:100000000C9446000C9463000C9463000C94630001
:100010000C9463000C9463000C9463000C946300D4
:100020000C9463000C9463000C9463000C946300C4
:100030000C9463000C9463000C9463000C946300B4
:100040000C9463000C9463000C9463000C946300A4
:100050000C9463000C9463000C9463000C94630094
:100060000C9463000C9463000C9463000C94630084
:100070000C9463000C9463000C9463000C94630074
:100080000C9463000C9463000C94630011241FBE55
:10009000CFEFD0E1DEBFCDBF12E0A0E0B1E0E0E8FD
:1000A000F2E800E00BBF02C007900D92A437B10741
:1000B000D9F713E0A4E7B2E001C01D92AA31B1075D
:1000C000E1F70C9465000C940000CF93DF93CDB75B
:1000D000DEB72C970FB6F894DEBF0FBECDBFEAE3B4
:1000E000F0E08FEF8083E7E3F0E08FEF8083E1E6DD
:1000F000F0E01082E8E3F0E01082E2E6F0E0108247
:1001000010920D0310920C03109205031092040339
:100110001092CB021092CA0281E090E09093CD023F
:100120008093CC0281E090E09093E7028093E60216
:100130001092D7021092D6021092D5021092D402D9
:100140000E940D1E0E941C1E80E090E0A0E7B1E41A
:100150008B839C83AD83BE8326E636E646E655E474
:100160006B817C818D819E810E944039DC01CB01B5
:1001700089879A87AB87BC8720E030E040E85FE35F
:1001800069857A858B859C850E94CA3A88230CF004
:1001900005C081E090E098878F831AC020E03FEF90
:1001A0004FE757E469857A858B859C850E945E3A86
:1001B00018160CF003C018861F820AC069857A855C
:1001C0008B859C850E948F37DC01CB0198878F83BC
:1001D0008F8198859A83898389819A810197F1F724
:1001E0009A8389830E949A2F0E94C1230E9486329B
:1001F0001092ED021092EC020DC080E090E00E949F
:10020000B60C8091EC029091ED0201969093ED0274
:100210008093EC028091EC029091ED028A3091057E
:1002200064F30E948B2F0E94351E81E090E00E94B3
:10023000B60C8091060390910703893C910514F058
:100240000E94BF1A8091DE029091DF028B3A9105E5
:10025000E4F480910E0390910F038B3A9105ACF476
:100260008091DC029091DD028E3691053CF4809104
:100270000003909101038E3691053CF081E090E0FF
:100280009093FD028093FC0204C01092FD02109234
:10029000FC028091DC029091DD028E36910574F4AF
:1002A00080910003909101038E3691053CF481E02A
:1002B00090E09093E1028093E00204C01092E1028A
:1002C0001092E0028091DE029091DF028B3A91055C
:1002D0003CF081E090E09093FF028093FE0204C026
:1002E0001092FF021092FE0280910E0390910F0374
:1002F0008B3A91053CF081E090E09093C9028093A5
:10030000C80204C01092C9021092C8028091100362
:100310009091110321E0853092077CF080910803D1
:100320009091090321E0853092073CF081E090E054
:1003300090930B0380930A0304C010920B03109256
:100340000A030E94A40171CF0F931F93CF93DF93F1
:10035000CDB7DEB7C05CD0400FB6F894DEBF0FBE9D
:10036000CDBF8091FC029091FD028130910509F092
:100370007DC08091E0029091E102009709F076C083
:100380008091FE029091FF02009709F06FC080916A
:10039000C8029091C902009709F068C080910A03D1
:1003A00090910B03009709F061C08091CC0290916D
:1003B000CD028130910509F03FC08091E602909115
:1003C000E70281309105C1F58091D6029091D70264
:1003D0008837910544F58091D4029091D5028837F1
:1003E00091050CF58091D6029091D7024E9690938C
:1003F000D7028093D6028091D4029091D5024E9676
:100400009093D5028093D4028091D6029091D70226
:100410002091D4023091D502BC01C9010E948E36D0
:100420000E94A81C23C068E770E088E790E00E9463
:100430008E360E94A81C1AC00E9414360E945136A3
:1004400081E090E09093CD028093CC0281E090E037
:100450009093E7028093E6021092D7021092D602A0
:100460001092D5021092D4020E94A81C8091FC0226
:100470009091FD02009709F078C08091E002909180
:10048000E1028130910509F070C080910A039091DA
:100490000B03009709F069C08091CC029091CD02C6
:1004A0008130910509F049C08091E6029091E70200
:1004B000009709F042C08091D6029091D7028A3508
:1004C000910594F58091D4029091D5028A359105D9
:1004D0005CF58091D6029091D7024E969093D70208
:1004E0008093D6028091D4029091D5024E9690933B
:1004F000D5028093D40281E090E09093CD02809366
:10050000CC021092E7021092E6028091D402909100
:10051000D5022091D6023091D702BC01C9010E94B8
:100520008C340E94A81C21C06AE570E08AE590E046
:100530000E948C340E94A81C18C00E9414360E948D
:10054000513681E090E09093CD028093CC021092DE
:10055000E7021092E6021092D7021092D602109291
:10056000D5021092D4020E94A81C8091FE029091A4
:10057000FF028130910509F07DC08091C802909101
:10058000C902009709F076C08091E0029091E102E3
:10059000009709F06FC080910A0390910B030097B8
:1005A00009F068C08091CC029091CD028130910514
:1005B00009F042C08091E6029091E7020097E1F5D0
:1005C0008091D6029091D7028837910504F58091E9
:1005D000D6029091D7024E969093D7028093D6027E
:1005E0001092D5021092D40281E090E09093CD0257
:1005F0008093CC021092E7021092E6028091D6021C
:100600009091D7020E9492350E94A81C33C010928C
:10061000D5021092D40281E090E09093CD028093B5
:10062000CC021092E7021092E60288E790E00E9466
:1006300092350E94A81C1EC08091CC029091CD02E0
:10064000009711F40E9414360E94513681E090E028
:100650009093CD028093CC021092E7021092E602B2
:100660001092D7021092D6021092D5021092D402A4
:100670000E94A81C8091C8029091C9028130910506
:1006800009F07DC08091FE029091FF02009709F071
:1006900076C08091E0029091E102009709F06FC06E
:1006A00080910A0390910B03009709F068C0809134
:1006B000CC029091CD02009709F043C08091E602F0
:1006C0009091E70281309105E1F58091D4029091FB
:1006D000D5028837910504F51092D7021092D60200
:1006E0008091D4029091D5024E969093D50280933A
:1006F000D4021092CD021092CC0281E090E090934F
:10070000E7028093E6028091D4029091D5020E9484
:1007100010350E94A81C33C01092D7021092D60246
:100720001092CD021092CC0281E090E09093E7020B
:100730008093E60288E790E00E9410350E94A81C92
:100740001EC08091E6029091E702009711F40E948A
:1007500051360E9414361092CD021092CC0281E0E4
:1007600090E09093E7028093E6021092D7021092F5
:10077000D6021092D5021092D4020E94A81C809139
:10078000FE029091FF028130910509F07FC08091B7
:10079000C8029091C9028130910509F077C080911B
:1007A000E0029091E102009709F070C080910A0385
:1007B00090910B03009709F069C08091CC02909151
:1007C000CD028130910509F049C08091E6029091F7
:1007D000E702009709F042C08091D6029091D702BB
:1007E0008A35910594F58091D4029091D5028A358D
:1007F00091055CF58091D6029091D7024E96909328
:10080000D7028093D6028091D4029091D5024E9661
:100810009093D5028093D40281E090E09093CD0232
:100820008093CC021092E7021092E6028091D402EB
:100830009091D5022091D6023091D702BC01C90116
:100840000E948C340E94A81C21C06AE570E08AE5F1
:1008500090E00E948C340E94A81C18C00E9414369C
:100860000E94513681E090E09093CD028093CC02BB
:100870001092E7021092E6021092D7021092D6026E
:100880001092D5021092D4020E94A81C80910A03F3
:1008900090910B038130910511F00C94AA0C0E94E9
:1008A00014360E94513681E090E09093CD028093FF
:1008B000CC0281E090E09093E7028093E6021092F0
:1008C000D7021092D6021092D5021092D4020E9442
:1008D000A81C0E948B2FFE01E954FF4F80E090E09E
:1008E000A0E8BFE380839183A283B3838E01035486
:1008F0001F4FFE01E954FF4F26E636E646E655E473
:1009000060817181828193810E944039DC01CB0139
:10091000F80180839183A283B383FE01E354FF4FE8
:1009200020E030E040E85FE3608171818281938163
:100930000E94CA3A88230CF008C0FE01E554FF4F1C
:1009400081E090E09183808327C0FE01E354FF4F54
:1009500020E03FEF4FE757E460817181828193810E
:100960000E945E3A18160CF006C0FE01E554FF4FD7
:100970001182108211C08E0105541F4FFE01E354F5
:10098000FF4F60817181828193810E948F37DC01EA
:10099000CB01F80191838083DE01AB54BF4FFE0190
:1009A000E554FF4F808191818D939C93FE01EB5420
:1009B000FF4F808191810197F1F7FE01EB54FF4FCA
:1009C0009183808363E070E081E090E00E9480305A
:1009D000FE01E555FF4F80E090E0A0E8BFE3808393
:1009E0009183A283B3838E010F541F4FFE01E555FF
:1009F000FF4F26E636E646E655E460817181828146
:100A000093810E944039DC01CB01F80180839183FE
:100A1000A283B383FE01EF54FF4F20E030E040E8B3
:100A20005FE360817181828193810E94CA3A882349
:100A30000CF008C0FE01E155FF4F81E090E091838A
:100A4000808327C0FE01EF54FF4F20E03FEF4FE7C8
:100A500057E460817181828193810E945E3A181609
:100A60000CF006C0FE01E155FF4F1182108211C04B
:100A70008E0101551F4FFE01EF54FF4F60817181C0
:100A8000828193810E948F37DC01CB01F801918331
:100A90008083DE01A755BF4FFE01E155FF4F8081E6
:100AA00091818D939C93FE01E755FF4F8081918149
:100AB0000197F1F7FE01E755FF4F9183808389E3AA
:100AC00091E00E945B30FE01E156FF4F80E090E034
:100AD000A0E8BFE380839183A283B3838E010B558B
:100AE0001F4FFE01E156FF4F26E636E646E655E487
:100AF00060817181828193810E944039DC01CB0148
:100B0000F80180839183A283B383FE01EB55FF4FED
:100B100020E030E040E85FE3608171818281938171
:100B20000E94CA3A88230CF008C0FE01ED55FF4F21
:100B300081E090E09183808327C0FE01EB55FF4F59
:100B400020E03FEF4FE757E460817181828193811C
:100B50000E945E3A18160CF006C0FE01ED55FF4FDC
:100B60001182108211C08E010D551F4FFE01EB55F1
:100B7000FF4F60817181828193810E948F37DC01F8
:100B8000CB01F80191838083DE01A356BF4FFE01A4
:100B9000ED55FF4F808191818D939C93FE01E3562B
:100BA000FF4F808191810197F1F7FE01E356FF4FDE
:100BB0009183808365E070E082E090E00E94803065
:100BC000FE01ED56FF4F80E090E0A0E8BFE3808398
:100BD0009183A283B3838E0107561F4FFE01ED560A
:100BE000FF4F26E636E646E655E460817181828154
:100BF00093810E944039DC01CB01F801808391830D
:100C0000A283B383FE01E756FF4F20E030E040E8C7
:100C10005FE360817181828193810E94CA3A882357
:100C20000CF008C0FE01E956FF4F81E090E091838F
:100C3000808327C0FE01E756FF4F20E03FEF4FE7DC
:100C400057E460817181828193810E945E3A181617
:100C50000CF006C0FE01E956FF4F1182108211C050
:100C60008E0109561F4FFE01E756FF4F60817181CB
:100C7000828193810E948F37DC01CB01F80191833F
:100C80008083DE01AF56BF4FFE01E956FF4F8081E2
:100C900091818D939C93FE01EF56FF4F808191814E
:100CA0000197F1F7FE01EF56FF4F9183808380E4B7
:100CB00091E00E945B300E941F1D8091E0029091A4
:100CC000E1028130910571F46EE170E08EE190E017
:100CD0000E9407340E94961D0E94961D0E941436A1
:100CE0000E9451361092ED021092EC0261C06EE14A
:100CF00070E08EE190E00E948C3480E090E00E94F1
:100D0000B60C0E941F1D6CE370E08CE390E00E9423
:100D10008C3480E090E00E94B60C0E941F1D80E0A1
:100D200090E00E94B60C0E941F1D80E090E00E949F
:100D3000B60C0E9414360E94513680E090E00E946A
:100D4000B60C0E941F1D6EE170E08EE190E00E94E3
:100D5000073480E090E00E94B60C0E941F1D6CE3F7
:100D600070E08CE390E00E94073480E090E00E9405
:100D7000B60C0E941F1D80E090E00E94B60C0E94FD
:100D80001F1D80E090E00E94B60C0E9414360E9465
:100D9000513680E090E00E94B60C0E941F1D8091A9
:100DA000EC029091ED0201969093ED028093EC029B
:100DB0008091EC029091ED02833091050CF497CF75
:100DC0008091100390911103853691050CF401C3B5
:100DD0008091080390910903853691050CF4F9C2BE
:100DE0000E948B2FFE01E957FF4F80E090E0A0E8C2
:100DF000BFE380839183A283B3838E0103571F4F88
:100E0000FE01E957FF4F26E636E646E655E46081E7
:100E10007181828193810E944039DC01CB01F8010C
:100E200080839183A283B383FE01E357FF4F20E0C9
:100E300030E040E85FE360817181828193810E94AC
:100E4000CA3A88230CF008C0FE01E557FF4F81E045
:100E500090E09183808327C0FE01E357FF4F20E09D
:100E60003FEF4FE757E460817181828193810E9457
:100E70005E3A18160CF006C0FE01E557FF4F1182CE
:100E8000108211C08E0105571F4FFE01E357FF4F1F
:100E900060817181828193810E948F37DC01CB0157
:100EA000F80191838083DE01AB57BF4FFE01E55708
:100EB000FF4F808191818D939C93FE01EB57FF4FF3
:100EC000808191810197F1F7FE01EB57FF4F9183EC
:100ED000808363E070E081E090E00E948030FE015A
:100EE000E558FF4F80E090E0A0E8BFE38083918366
:100EF000A283B3838E010F571F4FFE01E558FF4FAA
:100F000026E636E646E655E460817181828193816A
:100F10000E944039DC01CB01F80180839183A283D8
:100F2000B383FE01EF57FF4F20E030E040E85FE37E
:100F300060817181828193810E94CA3A88230CF07A
:100F400008C0FE01E158FF4F81E090E0918380836B
:100F500027C0FE01EF57FF4F20E03FEF4FE757E478
:100F600060817181828193810E945E3A18160CF033
:100F700006C0FE01E158FF4F1182108211C08E01A0
:100F800001581F4FFE01EF57FF4F60817181828131
:100F900093810E948F37DC01CB01F801918380831C
:100FA000DE01A758BF4FFE01E158FF4F80819181BC
:100FB0008D939C93FE01E758FF4F808191810197AB
:100FC000F1F7FE01E758FF4F918380838DE491E0B4
:100FD0000E945B30FE01E159FF4F80E090E0A0E805
:100FE000BFE380839183A283B3838E010B581F4F8D
:100FF000FE01E159FF4F26E636E646E655E46081FC
:101000007181828193810E944039DC01CB01F8011A
:1010100080839183A283B383FE01EB58FF4F20E0CE
:1010200030E040E85FE360817181828193810E94BA
:10103000CA3A88230CF008C0FE01ED58FF4F81E04A
:1010400090E09183808327C0FE01EB58FF4F20E0A2
:101050003FEF4FE757E460817181828193810E9465
:101060005E3A18160CF006C0FE01ED58FF4F1182D3
:10107000108211C08E010D581F4FFE01EB58FF4F1B
:1010800060817181828193810E948F37DC01CB0165
:10109000F80191838083DE01A359BF4FFE01ED5813
:1010A000FF4F808191818D939C93FE01E359FF4F07
:1010B000808191810197F1F7FE01E359FF4F918300
:1010C000808361E070E082E090E00E948030FE0169
:1010D000ED59FF4F80E090E0A0E8BFE3808391836B
:1010E000A283B3838E0107591F4FFE01ED59FF4FB5
:1010F00026E636E646E655E4608171818281938179
:101100000E944039DC01CB01F80180839183A283E6
:10111000B383FE01E759FF4F20E030E040E85FE392
:1011200060817181828193810E94CA3A88230CF088
:1011300008C0FE01E959FF4F81E090E09183808370
:1011400027C0FE01E759FF4F20E03FEF4FE757E48C
:1011500060817181828193810E945E3A18160CF041
:1011600006C0FE01E959FF4F1182108211C08E01A5
:1011700009591F4FFE01E759FF4F6081718182813C
:1011800093810E948F37DC01CB01F801918380832A
:10119000DE01AF59BF4FFE01E959FF4F80819181B8
:1011A0008D939C93FE01EF59FF4F808191810197B0
:1011B000F1F7FE01EF59FF4F918380838DE591E0B8
:1011C0000E945B300E941F1D0E941F1D0E941F1D58
:1011D0000E941F1D0E948B2FFE01E95AFF4F80E0E5
:1011E00090E0A0E8BFE380839183A283B3838E0164
:1011F000035A1F4FFE01E95AFF4F26E636E646E640
:1012000055E460817181828193810E944039DC01C3
:10121000CB01F80180839183A283B383FE01E35A5B
:10122000FF4F20E030E040E85FE360817181828120
:1012300093810E94CA3A88230CF008C0FE01E55A47
:10124000FF4F81E090E09183808327C0FE01E35A45
:10125000FF4F20E03FEF4FE757E4608171818281CB
:1012600093810E945E3A18160CF006C0FE01E55A02
:10127000FF4F1182108211C08E01055A1F4FFE01CF
:10128000E35AFF4F60817181828193810E948F3781
:10129000DC01CB01F80191838083DE01AB5ABF4FA3
:1012A000FE01E55AFF4F808191818D939C93FE0151
:1012B000EB5AFF4F808191810197F1F7FE01EB5AC4
:1012C000FF4F9183808363E070E081E090E00E94B3
:1012D0008030E8E3F0E081E38083FE01E55BFF4FCF
:1012E00080E090E0A0E8BFE380839183A283B38392
:1012F0008E010F5A1F4FFE01E55BFF4F26E636E6D3
:1013000046E655E460817181828193810E94403973
:10131000DC01CB01F80180839183A283B383FE01BA
:10132000EF5AFF4F20E030E040E85FE360817181D9
:10133000828193810E94CA3A88230CF008C0FE0182
:10134000E15BFF4F81E090E09183808327C0FE0145
:10135000EF5AFF4F20E03FEF4FE757E46081718184
:10136000828193810E945E3A18160CF006C0FE013D
:10137000E15BFF4F1182108211C08E01015B1F4F94
:10138000FE01EF5AFF4F60817181828193810E943B
:101390008F37DC01CB01F80191838083DE01A75BED
:1013A000BF4FFE01E15BFF4F808191818D939C9344
:1013B000FE01E75BFF4F808191810197F1F7FE010C
:1013C000E75BFF4F9183808380E791E00E945B3071
:1013D00078C10E948B2FFE01FF9680E090E0A0E88C
:1013E000BFE380839183A283B3838E010B5B1F4F86
:1013F000FE01FF9626E636E646E655E460817181F9
:10140000828193810E944039DC01CB01F801808305
:101410009183A283B383FE01EB5BFF4F20E030E0BA
:1014200040E85FE360817181828193810E94CA3AC2
:1014300088230CF008C0FE01ED5BFF4F81E090E0D7
:101440009183808327C0FE01EB5BFF4F20E03FEFDD
:101450004FE757E460817181828193810E945E3AF7
:1014600018160CF006C0FE01ED5BFF4F11821082D2
:1014700011C08E010D5B1F4FFE01EB5BFF4F6081C2
:101480007181828193810E948F37DC01CB01F80149
:1014900091838083FE01ED5BFF4F808191819EAF40
:1014A0008DAF8DAD9EAD0197F1F79EAF8DAF63E02F
:1014B00070E081E090E00E94803080E090E0A0E861
:1014C000BFE38BAB9CABADABBEAB26E636E646E6E8
:1014D00055E46BA97CA98DA99EA90E944039DC0125
:1014E000CB0189AF9AAFABAFBCAF20E030E040E8B2
:1014F0005FE369AD7AAD8BAD9CAD0E94CA3A88239B
:101500000CF005C081E090E098AF8FAB1AC020E0EE
:101510003FEF4FE757E469AD7AAD8BAD9CAD0E94CC
:101520005E3A18160CF003C018AE1FAA0AC069ADC7
:101530007AAD8BAD9CAD0E948F37DC01CB0198AFAB
:101540008FAB8FA998AD9AAB89AB89A99AA901975E
:10155000F1F79AAB89AB8CE791E00E945B3080E0B9
:1015600090E0A0E8BFE38FA398A7A9A7BAA726E6B3
:1015700036E646E655E46FA178A589A59AA50E94AE
:101580004039DC01CB018DA79EA7AFA7B8AB20E007
:1015900030E040E85FE36DA57EA58FA598A90E9485
:1015A000CA3A88230CF005C081E090E09CA78BA785
:1015B0001AC020E03FEF4FE757E46DA57EA58FA549
:1015C00098A90E945E3A18160CF003C01CA61BA630
:1015D0000AC06DA57EA58FA598A90E948F37DC0152
:1015E000CB019CA78BA78BA59CA59EA38DA38DA1AA
:1015F0009EA10197F1F79EA38DA365E070E082E0C4
:1016000090E00E94803080E090E0A0E8BFE38B8F04
:101610009C8FAD8FBE8F26E636E646E655E46B8D91
:101620007C8D8D8D9E8D0E944039DC01CB0189A37C
:101630009AA3ABA3BCA320E030E040E85FE369A13C
:101640007AA18BA19CA10E94CA3A88230CF005C004
:1016500081E090E098A38F8F1AC020E03FEF4FE722
:1016600057E469A17AA18BA19CA10E945E3A181649
:101670000CF003C018A21F8E0AC069A17AA18BA129
:101680009CA10E948F37DC01CB0198A38F8F8F8D97
:1016900098A19A8F898F898D9A8D0197F1F79A8FEA
:1016A000898F88E891E00E945B300E9414360E9486
:1016B00051360E941F1D0E941F1D0E941F1D0E9467
:1016C0001F1D6EE170E08EE190E00E9413370E94D2
:1016D000A81C0E94961D6CE370E08CE390E00E94D1
:1016E00013370E94A81C0E94961D6AE570E08AE5E7
:1016F00090E00E9413370E94A81C0E94961D6AE584
:1017000070E08AE590E00E9413370E94A81C0E94B6
:101710001F1D0E941F1D0E941F1D0E941F1DE8E328
:10172000F0E081E080830E9414360E9451360E94CE
:10173000961D0E94961D6EE170E08EE190E00E9481
:1017400007340E94A81C0E94961D6CE370E08CE395
:1017500090E00E9407340E94A81C0E94961D6AE532
:1017600070E08AE590E00E9407340E94A81C0E9465
:10177000961D6AE570E08AE590E00E9407340E94B9
:101780001F1D0E941F1D0E941F1D0E941F1D0E94E1
:101790001F1D0E941F1D0E9414360E9451360E9478
:1017A000A81C1092110310921003109209031092BA
:1017B00008031092CF021092CE021FC08091CE0279
:1017C0009091CF02880F991FFC01EC58FD4F1182B8
:1017D00010828091CE029091CF02880F991FFC0158
:1017E000E857FD4F118210828091CE029091CF0276
:1017F00001969093CF028093CE028091CE02909179
:10180000CF028A309105D4F20E948B2F80E090E0C5
:10181000A0E8BFE38F87988BA98BBA8B26E636E6C4
:1018200046E655E46F85788989899A890E9440390E
:10183000DC01CB018D8B9E8BAF8BB88F20E030E02D
:1018400040E85FE36D897E898F89988D0E94CA3A4E
:1018500088230CF005C081E090E09C8B8B8B1AC034
:1018600020E03FEF4FE757E46D897E898F89988D9F
:101870000E945E3A18160CF003C01C8A1B8A0AC02C
:101880006D897E898F89988D0E948F37DC01CB010D
:101890009C8B8B8B8B899C899E878D878D859E8564
:1018A0000197F1F79E878D8760E070E080E090E01F
:1018B0000E94803080E090E0A0E8BFE38B839C83AF
:1018C000AD83BE8326E636E646E655E46B817C8131
:1018D0008D819E810E944039DC01CB0189879A87E6
:1018E000AB87BC8720E030E040E85FE369857A851C
:1018F0008B859C850E94CA3A88230CF005C081E044
:1019000090E098878F831AC020E03FEF4FE757E4BD
:1019100069857A858B859C850E945E3A18160CF045
:1019200003C018861F820AC069857A858B859C85CD
:101930000E948F37DC01CB0198878F838F81988538
:101940009A83898389819A810197F1F79A838983A0
:101950000E94351EC054DF4F0FB6F894DEBF0FBE95
:10196000CDBFDF91CF911F910F9108950F931F93DA
:10197000CF93DF93CDB7DEB7CA53D1400FB6F894FB
:10198000DEBF0FBECDBFFE01E75CFE4F91838083BB
:10199000E7E2F0E084E68083FE01E15DFE4F80E057
:1019A00090E0A0EAB0E480839183A283B3838E01A8
:1019B0000B5C1E4FFE01E15DFE4F26E636E646E675
:1019C00055E460817181828193810E944039DC01FC
:1019D000CB01F80180839183A283B383FE01EB5C8A
:1019E000FE4F20E030E040E85FE36081718182815A
:1019F00093810E94CA3A88230CF008C0FE01ED5C76
:101A0000FE4F81E090E09183808327C0FE01EB5C74
:101A1000FE4F20E03FEF4FE757E460817181828104
:101A200093810E945E3A18160CF006C0FE01ED5C30
:101A3000FE4F1182108211C08E010D5C1E4FFE01FF
:101A4000EB5CFE4F60817181828193810E948F37B0
:101A5000DC01CB01F80191838083DE01A35DBE4FE1
:101A6000FE01ED5CFE4F808191818D939C93FE0180
:101A7000E35DFE4F808191810197F1F7FE01E35D07
:101A8000FE4F91838083E5E2F0E080819927909377
:101A9000DB028093DA028091DA029091DB0290936C
:101AA000D9028093D8028091D8029091D902909364
:101AB000070380930603FE01ED5DFE4F80E090E09A
:101AC000A0EAB0E480839183A283B3838E01075D93
:101AD0001E4FFE01ED5DFE4F26E636E646E655E476
:101AE00060817181828193810E944039DC01CB0148
:101AF000F80180839183A283B383FE01E75DFE4FEB
:101B000020E030E040E85FE3608171818281938171
:101B10000E94CA3A88230CF008C0FE01E95DFE4F1E
:101B200081E090E09183808327C0FE01E75DFE4F56
:101B300020E03FEF4FE757E460817181828193811C
:101B40000E945E3A18160CF006C0FE01E95DFE4FD9
:101B50001182108211C08E01095D1E4FFE01E75DEA
:101B6000FE4F60817181828193810E948F37DC01F9
:101B7000CB01F80191838083DE01AF5DBE4FFE0192
:101B8000E95DFE4F808191818D939C93FE01EF5D15
:101B9000FE4F808191810197F1F7FE01EF5DFE4FCD
:101BA00091838083E7E2F0E083E68083FE01E95ED3
:101BB000FE4F80E090E0A0EAB0E480839183A283AE
:101BC000B3838E01035E1E4FFE01E95EFE4F26E6E3
:101BD00036E646E655E460817181828193810E94F8
:101BE0004039DC01CB01F80180839183A283B38368
:101BF000FE01E35EFE4F20E030E040E85FE36081FD
:101C00007181828193810E94CA3A88230CF008C0B6
:101C1000FE01E55EFE4F81E090E09183808327C066
:101C2000FE01E35EFE4F20E03FEF4FE757E46081A7
:101C30007181828193810E945E3A18160CF006C071
:101C4000FE01E55EFE4F1182108211C08E01055E1D
:101C50001E4FFE01E35EFE4F6081718182819381A0
:101C60000E948F37DC01CB01F80191838083DE0174
:101C7000AB5EBE4FFE01E55EFE4F808191818D938C
:101C80009C93FE01EB5EFE4F808191810197F1F7FD
:101C9000FE01EB5EFE4F91838083E5E2F0E0808100
:101CA00099279093DB028093DA028091DA02909177
:101CB000DB028C599F4F9093DB028093DA02809174
:101CC000DA029091DB029093D9028093D80280913E
:101CD000D8029091D9029093DF028093DE02E7E26E
:101CE000F0E082E68083FE01E55FFE4F80E090E059
:101CF000A0EAB0E480839183A283B3838E010F5E58
:101D00001E4FFE01E55FFE4F26E636E646E655E449
:101D100060817181828193810E944039DC01CB0115
:101D2000F80180839183A283B383FE01EF5EFE4FAF
:101D300020E030E040E85FE360817181828193813F
:101D40000E94CA3A88230CF008C0FE01E15FFE4FF2
:101D500081E090E09183808327C0FE01EF5EFE4F1B
:101D600020E03FEF4FE757E46081718182819381EA
:101D70000E945E3A18160CF006C0FE01E15FFE4FAD
:101D80001182108211C08E01015F1E4FFE01EF5EB5
:101D9000FE4F60817181828193810E948F37DC01C7
:101DA000CB01F80191838083DE01A75FBE4FFE0166
:101DB000E15FFE4F808191818D939C93FE01E75FEF
:101DC000FE4F808191810197F1F7FE01E75FFE4FA1
:101DD00091838083E5E2F0E0808199279093DB0294
:101DE0008093DA028091DA029091DB028C599F4F46
:101DF0009093DB028093DA028091DA029091DB0209
:101E00009093D9028093D8028091D8029091D90200
:101E100090930F0380930E03E7E2F0E086E6808361
:101E2000FE01E150FF4F80E090E0A0EAB0E4808343
:101E30009183A283B3838E010B5F1E4FFE01E1509D
:101E4000FF4F26E636E646E655E4608171818281E1
:101E500093810E944039DC01CB01F801808391839A
:101E6000A283B383FE01EB5FFE4F20E030E040E849
:101E70005FE360817181828193810E94CA3A8823E5
:101E80000CF008C0FE01ED5FFE4F81E090E0918311
:101E9000808327C0FE01EB5FFE4F20E03FEF4FE75E
:101EA00057E460817181828193810E945E3A1816A5
:101EB0000CF006C0FE01ED5FFE4F1182108211C0D2
:101EC0008E010D5F1E4FFE01EB5FFE4F6081718141
:101ED000828193810E948F37DC01CB01F8019183CD
:101EE0008083DE01A350BF4FFE01ED5FFE4F808176
:101EF00091818D939C93FE01E350FF4F80819181EE
:101F00000197F1F7FE01E350FF4F91838083E5E2F3
:101F1000F0E0808199279093DB028093DA02809130
:101F2000DA029091DB028C599F4F9093DB028093F1
:101F3000DA0280910C0390910D032091DA02309126
:101F4000DB02880F991FFC01EC58FD4F3183208381
:101F5000E7E2F0E085E68083FE01ED50FF4F80E090
:101F600090E0A0EAB0E480839183A283B3838E01E2
:101F700007501F4FFE01ED50FF4F26E636E646E6BE
:101F800055E460817181828193810E944039DC0136
:101F9000CB01F80180839183A283B383FE01E750D4
:101FA000FF4F20E030E040E85FE360817181828193
:101FB00093810E94CA3A88230CF008C0FE01E950C0
:101FC000FF4F81E090E09183808327C0FE01E750BE
:101FD000FF4F20E03FEF4FE757E46081718182813E
:101FE00093810E945E3A18160CF006C0FE01E9507B
:101FF000FF4F1182108211C08E0109501F4FFE0148
:10200000E750FF4F60817181828193810E948F37F9
:10201000DC01CB01F80191838083DE01AF50BF4F1B
:10202000FE01E950FF4F808191818D939C93FE01C9
:10203000EF50FF4F808191810197F1F7FE01EF5042
:10204000FF4F91838083E5E2F0E0808199279093B0
:10205000DB028093DA028091DA029091DB028C59E4
:102060009F4F9093DB028093DA0280910C03909152
:102070000D032091DA023091DB02880F991FFC01D9
:10208000E857FD4F31832083E7E2F0E081E680836B
:10209000FE01E951FF4F80E090E0A0EAB0E48083C8
:1020A0009183A283B3838E0103511F4FFE01E95137
:1020B000FF4F26E636E646E655E46081718182816F
:1020C00093810E944039DC01CB01F8018083918328
:1020D000A283B383FE01E351FF4F20E030E040E8EC
:1020E0005FE360817181828193810E94CA3A882373
:1020F0000CF008C0FE01E551FF4F81E090E09183B4
:10210000808327C0FE01E351FF4F20E03FEF4FE700
:1021100057E460817181828193810E945E3A181632
:102120000CF006C0FE01E551FF4F1182108211C074
:102130008E0105511F4FFE01E351FF4F60817181F8
:10214000828193810E948F37DC01CB01F80191835A
:102150008083DE01AB51BF4FFE01E551FF4F80810F
:1021600091818D939C93FE01EB51FF4F8081918172
:102170000197F1F7FE01EB51FF4F91838083E5E278
:10218000F0E0808199279093DB028093DA028091BE
:10219000DA029091DB028C599F4F9093D902809381
:1021A000D80280910C0390910D032091D8023091B8
:1021B000D902880F991FFC01E456FD4F318320831B
:1021C000E7E2F0E080E68083FE01E552FF4F80E029
:1021D00090E0A0EAB0E480839183A283B3838E0170
:1021E0000F511F4FFE01E552FF4F26E636E646E649
:1021F00055E460817181828193810E944039DC01C4
:10220000CB01F80180839183A283B383FE01EF5158
:10221000FF4F20E030E040E85FE360817181828120
:1022200093810E94CA3A88230CF008C0FE01E15253
:10223000FF4F81E090E09183808327C0FE01EF5142
:10224000FF4F20E03FEF4FE757E4608171818281CB
:1022500093810E945E3A18160CF006C0FE01E1520E
:10226000FF4F1182108211C08E0101521F4FFE01DB
:10227000EF51FF4F60817181828193810E948F377E
:10228000DC01CB01F80191838083DE01A752BF4FAF
:10229000FE01E152FF4F8081918111969C938E93B4
:1022A000FE01E752FF4F808191810197F1F7FE0116
:1022B000E752FF4F91838083E5E2F0E08081992728
:1022C0009093DB028093DA028091DA029091DB0234
:1022D0008C599F4F9093D9028093D80280910C0320
:1022E00090910D032091D8023091D902880F991F47
:1022F000FC01E055FD4F31832083FE01E75CFE4F7A
:10230000808191818130910511F00C94D9198091CF
:10231000DE029091DF029F938F9386E991E09F9375
:102320008F9388EF92E09F938F930E947A3D8DB7B1
:102330009EB706960FB6F8949EBF0FBE8DBFFE01E6
:10234000E153FF4F80E090E0A0EAB0E48083918306
:10235000A283B3838E010B521F4FFE01E153FF4F47
:1023600026E636E646E655E46081718182819381F6
:102370000E944039DC01CB01F80180839183A28364
:10238000B383FE01EB52FF4F20E030E040E85FE313
:1023900060817181828193810E94CA3A88230CF006
:1023A00008C0FE01ED52FF4F81E090E091838083F1
:1023B00027C0FE01EB52FF4F20E03FEF4FE757E40D
:1023C00060817181828193810E945E3A18160CF0BF
:1023D00006C0FE01ED52FF4F1182108211C08E0126
:1023E0000D521F4FFE01EB52FF4F608171818281C0
:1023F00093810E948F37DC01CB01F80191838083A8
:10240000DE01A353BF4FFE01ED52FF4F808191814A
:102410008D939C93FE01E353FF4F8081918101973F
:10242000F1F7FE01E353FF4F9183808365E070E095
:1024300082E090E00E948030FE01ED53FF4F80E08B
:1024400090E0A0EAB0E480839183A283B3838E01FD
:1024500007531F4FFE01ED53FF4F26E636E646E6D3
:1024600055E460817181828193810E944039DC0151
:10247000CB01F80180839183A283B383FE01E753EC
:10248000FF4F20E030E040E85FE3608171818281AE
:1024900093810E94CA3A88230CF008C0FE01E953D8
:1024A000FF4F81E090E09183808327C0FE01E753D6
:1024B000FF4F20E03FEF4FE757E460817181828159
:1024C00093810E945E3A18160CF006C0FE01E95393
:1024D000FF4F1182108211C08E0109531F4FFE0160
:1024E000E753FF4F60817181828193810E948F3712
:1024F000DC01CB01F80191838083DE01AF53BF4F34
:10250000FE01E953FF4F808191818D939C93FE01E1
:10251000EF53FF4F808191810197F1F7FE01EF5357
:10252000FF4F9183808388EF92E00E945B30FE0131
:10253000E954FF4F80E090E0A0EAB0E4808391830B
:10254000A283B3838E0103541F4FFE01E954FF4F52
:1025500026E636E646E655E4608171818281938104
:102560000E944039DC01CB01F80180839183A28372
:10257000B383FE01E354FF4F20E030E040E85FE327
:1025800060817181828193810E94CA3A88230CF014
:1025900008C0FE01E554FF4F81E090E09183808305
:1025A00027C0FE01E354FF4F20E03FEF4FE757E421
:1025B00060817181828193810E945E3A18160CF0CD
:1025C00006C0FE01E554FF4F1182108211C08E013A
:1025D00005541F4FFE01E354FF4F608171818281DA
:1025E00093810E948F37DC01CB01F80191838083B6
:1025F000DE01AB54BF4FFE01E554FF4F8081918156
:102600008D939C93FE01EB54FF4F80819181019744
:10261000F1F7FE01EB54FF4F9183808380910E030D
:1026200090910F039F938F9386E991E09F938F93EF
:1026300088EE92E09F938F930E947A3D8DB79EB76C
:1026400006960FB6F8949EBF0FBE8DBFFE01E555EE
:10265000FF4F80E090E0A0EAB0E480839183A28302
:10266000B3838E010F541F4FFE01E555FF4F26E641
:1026700036E646E655E460817181828193810E944D
:102680004039DC01CB01F80180839183A283B383BD
:10269000FE01EF54FF4F20E030E040E85FE360814F
:1026A0007181828193810E94CA3A88230CF008C00C
:1026B000FE01E155FF4F81E090E09183808327C0C8
:1026C000FE01EF54FF4F20E03FEF4FE757E46081FA
:1026D0007181828193810E945E3A18160CF006C0C7
:1026E000FE01E155FF4F1182108211C08E0101558C
:1026F0001F4FFE01EF54FF4F6081718182819381F2
:102700000E948F37DC01CB01F80191838083DE01C9
:10271000A755BF4FFE01E155FF4F808191818D93F9
:102720009C93FE01E755FF4F808191810197F1F75E
:10273000FE01E755FF4F918380836FE070E082E0F8
:1027400090E00E948030FE01E156FF4F80E090E073
:10275000A0EAB0E480839183A283B3838E010B55FA
:102760001F4FFE01E156FF4F26E636E646E655E4EA
:1027700060817181828193810E944039DC01CB01AB
:10278000F80180839183A283B383FE01EB55FF4F51
:1027900020E030E040E85FE36081718182819381D5
:1027A0000E94CA3A88230CF008C0FE01ED55FF4F85
:1027B00081E090E09183808327C0FE01EB55FF4FBD
:1027C00020E03FEF4FE757E4608171818281938180
:1027D0000E945E3A18160CF006C0FE01ED55FF4F40
:1027E0001182108211C08E010D551F4FFE01EB5555
:1027F000FF4F60817181828193810E948F37DC015C
:10280000CB01F80191838083DE01A356BF4FFE0107
:10281000ED55FF4F808191818D939C93FE01E3568E
:10282000FF4F808191810197F1F7FE01E356FF4F41
:102830009183808388EE92E00E945B30FE01ED562A
:10284000FF4F80E090E0A0EAB0E480839183A28310
:10285000B3838E0107561F4FFE01ED56FF4F26E64C
:1028600036E646E655E460817181828193810E945B
:102870004039DC01CB01F80180839183A283B383CB
:10288000FE01E756FF4F20E030E040E85FE3608163
:102890007181828193810E94CA3A88230CF008C01A
:1028A000FE01E956FF4F81E090E09183808327C0CD
:1028B000FE01E756FF4F20E03FEF4FE757E460810E
:1028C0007181828193810E945E3A18160CF006C0D5
:1028D000FE01E956FF4F1182108211C08E01095688
:1028E0001F4FFE01E756FF4F608171818281938106
:1028F0000E948F37DC01CB01F80191838083DE01D8
:10290000AF56BF4FFE01E956FF4F808191818D93F5
:102910009C93FE01EF56FF4F808191810197F1F763
:10292000FE01EF56FF4F91838083809110039091B9
:1029300011039F938F9386E991E09F938F9384EF88
:1029400092E09F938F930E947A3D8DB79EB7069633
:102950000FB6F8949EBF0FBE8DBFFE01E957FF4F23
:1029600080E090E0A0EAB0E480839183A283B38307
:102970008E0103571F4FFE01E957FF4F26E636E64B
:1029800046E655E460817181828193810E944039DD
:10299000DC01CB01F80180839183A283B383FE0124
:1029A000E357FF4F20E030E040E85FE36081718152
:1029B000828193810E94CA3A88230CF008C0FE01EC
:1029C000E557FF4F81E090E09183808327C0FE01AF
:1029D000E357FF4F20E03FEF4FE757E460817181FD
:1029E000828193810E945E3A18160CF006C0FE01A7
:1029F000E557FF4F1182108211C08E0105571F4FFE
:102A0000FE01E357FF4F60817181828193810E94B3
:102A10008F37DC01CB01F80191838083DE01AB5756
:102A2000BF4FFE01E557FF4F808191818D939C93AD
:102A3000FE01EB57FF4F808191810197F1F7FE0175
:102A4000EB57FF4F9183808365E070E081E090E079
:102A50000E948030FE01E558FF4F80E090E0A0EA40
:102A6000B0E480839183A283B3838E010F571F4FFD
:102A7000FE01E558FF4F26E636E646E655E460815E
:102A80007181828193810E944039DC01CB01F80180
:102A900080839183A283B383FE01EF57FF4F20E031
:102AA00030E040E85FE360817181828193810E9420
:102AB000CA3A88230CF008C0FE01E158FF4F81E0BC
:102AC00090E09183808327C0FE01EF57FF4F20E005
:102AD0003FEF4FE757E460817181828193810E94CB
:102AE0005E3A18160CF006C0FE01E158FF4F118245
:102AF000108211C08E0101581F4FFE01EF57FF4F8A
:102B000060817181828193810E948F37DC01CB01CA
:102B1000F80191838083DE01A758BF4FFE01E15881
:102B2000FF4F808191818D939C93FE01E758FF4F69
:102B3000808191810197F1F7FE01E758FF4F918362
:102B4000808384EF92E00E945B30FE01E159FF4FE9
:102B500080E090E0A0EAB0E480839183A283B38315
:102B60008E010B581F4FFE01E159FF4F26E636E656
:102B700046E655E460817181828193810E944039EB
:102B8000DC01CB01F80180839183A283B383FE0132
:102B9000EB58FF4F20E030E040E85FE36081718157
:102BA000828193810E94CA3A88230CF008C0FE01FA
:102BB000ED58FF4F81E090E09183808327C0FE01B4
:102BC000EB58FF4F20E03FEF4FE757E46081718102
:102BD000828193810E945E3A18160CF006C0FE01B5
:102BE000ED58FF4F1182108211C08E010D581F4FFA
:102BF000FE01EB58FF4F60817181828193810E94B9
:102C00008F37DC01CB01F80191838083DE01A3596A
:102C1000BF4FFE01ED58FF4F808191818D939C93B2
:102C2000FE01E359FF4F808191810197F1F7FE0189
:102C3000E359FF4F918380838091080390910903AA
:102C40009F938F9386E991E09F938F9380ED92E01D
:102C50009F938F930E947A3D8DB79EB706960FB6CD
:102C6000F8949EBF0FBE8DBFFE01ED59FF4F80E06F
:102C700090E0A0EAB0E480839183A283B3838E01C5
:102C800007591F4FFE01ED59FF4F26E636E646E68F
:102C900055E460817181828193810E944039DC0119
:102CA000CB01F80180839183A283B383FE01E759AE
:102CB000FF4F20E030E040E85FE360817181828176
:102CC00093810E94CA3A88230CF008C0FE01E9599A
:102CD000FF4F81E090E09183808327C0FE01E75998
:102CE000FF4F20E03FEF4FE757E460817181828121
:102CF00093810E945E3A18160CF006C0FE01E95955
:102D0000FF4F1182108211C08E0109591F4FFE0121
:102D1000E759FF4F60817181828193810E948F37D3
:102D2000DC01CB01F80191838083DE01AF59BF4FF5
:102D3000FE01E959FF4F808191818D939C93FE01A3
:102D4000EF59FF4F808191810197F1F7FE01EF5913
:102D5000FF4F918380836FE070E081E090E00E94FC
:102D60008030FE01E95AFF4F80E090E0A0EAB0E435
:102D700080839183A283B3838E01035A1F4FFE0188
:102D8000E95AFF4F26E636E646E655E46081718152
:102D9000828193810E944039DC01CB01F80180835C
:102DA0009183A283B383FE01E35AFF4F20E030E01A
:102DB00040E85FE360817181828193810E94CA3A19
:102DC00088230CF008C0FE01E55AFF4F81E090E037
:102DD0009183808327C0FE01E35AFF4F20E03FEF3D
:102DE0004FE757E460817181828193810E945E3A4E
:102DF00018160CF006C0FE01E55AFF4F1182108232
:102E000011C08E01055A1F4FFE01E35AFF4F60812A
:102E10007181828193810E948F37DC01CB01F8019F
:102E200091838083DE01AB5ABF4FFE01E55AFF4F0D
:102E3000808191818D939C93FE01EB5AFF4F80819D
:102E400091810197F1F7FE01EB5AFF4F9183808347
:102E500080ED92E00E945B30FE01E55BFF4F80E079
:102E600090E0A0EAB0E480839183A283B3838E01D3
:102E70000F5A1F4FFE01E55BFF4F26E636E646E69A
:102E800055E460817181828193810E944039DC0127
:102E9000CB01F80180839183A283B383FE01EF5AB3
:102EA000FF4F20E030E040E85FE360817181828184
:102EB00093810E94CA3A88230CF008C0FE01E15BAE
:102EC000FF4F81E090E09183808327C0FE01EF5A9D
:102ED000FF4F20E03FEF4FE757E46081718182812F
:102EE00093810E945E3A18160CF006C0FE01E15B69
:102EF000FF4F1182108211C08E01015B1F4FFE0136
:102F0000EF5AFF4F60817181828193810E948F37D8
:102F1000DC01CB01F80191838083DE01A75BBF4F09
:102F2000FE01E15BFF4F808191818D939C93FE01B7
:102F3000E75BFF4F808191810197F1F7FE01E75B2D
:102F4000FF4F918380838091DC029091DD029F93FB
:102F50008F9386E991E09F938F9380EF92E09F9308
:102F60008F930E947A3D8DB79EB706960FB6F89460
:102F70009EBF0FBE8DBFFE01FF9680E090E0A0EAED
:102F8000B0E480839183A283B3838E010B5B1F4FD8
:102F9000FE01FF9626E636E646E655E4608171813D
:102FA000828193810E944039DC01CB01F80180834A
:102FB0009183A283B383FE01EB5BFF4F20E030E0FF
:102FC00040E85FE360817181828193810E94CA3A07
:102FD00088230CF008C0FE01ED5BFF4F81E090E01C
:102FE0009183808327C0FE01EB5BFF4F20E03FEF22
:102FF0004FE757E460817181828193810E945E3A3C
:1030000018160CF006C0FE01ED5BFF4F1182108216
:1030100011C08E010D5B1F4FFE01EB5BFF4F608106
:103020007181828193810E948F37DC01CB01F8018D
:1030300091838083FE01ED5BFF4F808191819EAF84
:103040008DAF8DAD9EAD0197F1F79EAF8DAF65E071
:1030500070E083E090E00E94803080E090E0A0EAA1
:10306000B0E48BAB9CABADABBEAB26E636E646E63A
:1030700055E46BA97CA98DA99EA90E944039DC0169
:10308000CB0189AF9AAFABAFBCAF20E030E040E8F6
:103090005FE369AD7AAD8BAD9CAD0E94CA3A8823DF
:1030A0000CF005C081E090E098AF8FAB1AC020E033
:1030B0003FEF4FE757E469AD7AAD8BAD9CAD0E9411
:1030C0005E3A18160CF003C018AE1FAA0AC069AD0C
:1030D0007AAD8BAD9CAD0E948F37DC01CB0198AFF0
:1030E0008FAB8FA998AD9AAB89AB89A99AA90197A3
:1030F000F1F79AAB89AB80EF92E00E945B3080E001
:1031000090E0A0EAB0E48FA398A7A9A7BAA726E603
:1031100036E646E655E46FA178A589A59AA50E94F2
:103120004039DC01CB018DA79EA7AFA7B8AB20E04B
:1031300030E040E85FE36DA57EA58FA598A90E94C9
:10314000CA3A88230CF005C081E090E09CA78BA7C9
:103150001AC020E03FEF4FE757E46DA57EA58FA58D
:1031600098A90E945E3A18160CF003C01CA61BA674
:103170000AC06DA57EA58FA598A90E948F37DC0196
:10318000CB019CA78BA78BA59CA59EA38DA38DA1EE
:103190009EA10197F1F79EA38DA3809100039091CA
:1031A00001039F938F9386E991E09F938F9382EE23
:1031B00092E09F938F930E947A3D8DB79EB70696BB
:1031C0000FB6F8949EBF0FBE8DBF80E090E0A0EADE
:1031D000B0E48B8F9C8FAD8FBE8F26E636E646E639
:1031E00055E46B8D7C8D8D8D9E8D0E944039DC0168
:1031F000CB0189A39AA3ABA3BCA320E030E040E8B5
:103200005FE369A17AA18BA19CA10E94CA3A88239D
:103210000CF005C081E090E098A38F8F1AC020E0E9
:103220003FEF4FE757E469A17AA18BA19CA10E94CF
:103230005E3A18160CF003C018A21F8E0AC069A1CE
:103240007AA18BA19CA10E948F37DC01CB0198A3AE
:103250008F8F8F8D98A19A8F898F898D9A8D0197E5
:10326000F1F79A8F898F6FE070E083E090E00E9421
:10327000803080E090E0A0EAB0E48F87988BA98B43
:10328000BA8B26E636E646E655E46F857889898965
:103290009A890E944039DC01CB018D8B9E8BAF8BCC
:1032A000B88F20E030E040E85FE36D897E898F8948
:1032B000988D0E94CA3A88230CF005C081E090E006
:1032C0009C8B8B8B1AC020E03FEF4FE757E46D8952
:1032D0007E898F89988D0E945E3A18160CF003C083
:1032E0001C8A1B8A0AC06D897E898F89988D0E94ED
:1032F0008F37DC01CB019C8B8B8B8B899C899E87C4
:103300008D878D859E850197F1F79E878D8782EE4B
:1033100092E00E945B3080E090E0A0EAB0E48B8312
:103320009C83AD83BE8326E636E646E655E46B8194
:103330007C818D819E810E944039DC01CB0189878F
:103340009A87AB87BC8720E030E040E85FE369857F
:103350007A858B859C850E94CA3A88230CF005C02B
:1033600081E090E098878F831AC020E03FEF4FE71D
:1033700057E469857A858B859C850E945E3A18168C
:103380000CF003C018861F820AC069857A858B8578
:103390009C850E948F37DC01CB0198878F838F81BA
:1033A00098859A83898389819A810197F1F79A8315
:1033B000898380910C0390910D03019690930D03E6
:1033C00080930C0380910C0390910D038A3091053A
:1033D00024F010920D0310920C038091120390912F
:1033E00013030196909313038093120380911203A9
:1033F000909113038530910524F0109213031092DD
:1034000012031092150310921403109219031092D4
:10341000180310920503109204031092CB0210922D
:10342000CA021092C7021092C6025DC08091C60205
:103430009091C702880F991FFC01EC58FD4F208125
:1034400031818091140390911503820F931F909303
:103450001503809314038091C6029091C702880FD0
:10346000991FFC01E857FD4F20813181809118039D
:1034700090911903820F931F90931903809318035F
:103480008091C6029091C702880F991FFC01E456F3
:10349000FD4F208131818091040390910503820FBB
:1034A000931F90930503809304038091C60290912B
:1034B000C702880F991FFC01E055FD4F2081318123
:1034C0008091CA029091CB02820F931F9093CB02FE
:1034D0008093CA028091C6029091C7020196909390
:1034E000C7028093C6028091C6029091C7028A30BB
:1034F00091050CF49BCF80911403909115032AE061
:1035000030E0B9010E94C040CB0190931103809339
:10351000100380911803909119032AE030E0B9015B
:103520000E94C040CB0190930903809308038091CF
:103530000403909105032AE030E0B9010E94C040E5
:10354000CB019093DD028093DC028091CA029091BE
:10355000CB022AE030E0B9010E94C040CB01909339
:10356000010380930003C65CDE4F0FB6F894DEBF04
:103570000FBECDBFDF91CF911F910F910895CF93D3
:10358000DF93CDB7DEB7E0970FB6F894DEBF0FBE7E
:10359000CDBF0E9414360E94513681E090E0909396
:1035A000CD028093CC0281E090E09093E70280937B
:1035B000E6021092D7021092D6021092D502109213
:1035C000D4020E94A81C0E948B2F80E090E0A0E80B
:1035D000BFE38FA398A7A9A7BAA726E636E646E6D3
:1035E00055E46FA178A589A59AA50E944039DC0110
:1035F000CB018DA79EA7AFA7B8AB20E030E040E895
:103600005FE36DA57EA58FA598A90E94CA3A88237D
:103610000CF005C081E090E09CA78BA71AC020E0C9
:103620003FEF4FE757E46DA57EA58FA598A90E94AF
:103630005E3A18160CF003C01CA61BA60AC06DA5A6
:103640007EA58FA598A90E948F37DC01CB019CA78E
:103650008BA78BA59CA59EA38DA38DA19EA1019751
:10366000F1F79EA38DA363E070E081E090E00E94FB
:10367000803080E090E0A0E8BFE38B8F9C8FAD8F1F
:10368000BE8F26E636E646E655E46B8D7C8D8D8D45
:103690009E8D0E944039DC01CB0189A39AA3ABA384
:1036A000BCA320E030E040E85FE369A17AA18BA1F0
:1036B0009CA10E94CA3A88230CF005C081E090E0EA
:1036C00098A38F8F1AC020E03FEF4FE757E469A11E
:1036D0007AA18BA19CA10E945E3A18160CF003C03F
:1036E00018A21F8E0AC069A17AA18BA19CA10E9479
:1036F0008F37DC01CB0198A38F8F8F8D98A19A8F84
:10370000898F898D9A8D0197F1F79A8F898F89E931
:1037100091E00E945B306EE170E08EE190E00E94EB
:1037200013370E94A81C0E94961D6CE370E08CE386
:1037300090E00E9413370E94A81C0E94961D6AE523
:1037400070E08AE590E00E9413370E94A81C0E9456
:10375000961D6AE570E08AE590E00E9413370E94AA
:10376000A81C0E941F1D0E941F1D0E941F1D0E9459
:103770001F1D0E9414360E9451360E94961D0E9401
:10378000961D6EE170E08EE190E00E9407340E9489
:10379000A81C0E94961D6CE370E08CE390E00E94F0
:1037A00007340E94A81C0E94961D6AE570E08AE515
:1037B00090E00E9407340E94A81C0E94961D6AE5B2
:1037C00070E08AE590E00E9407340E941F1D0E946D
:1037D0001F1D0E941F1D0E941F1D0E941F1D0E9471
:1037E0001F1D0E9414360E9451360E94A81C0E9480
:1037F000961D0E948B2F80E090E0A0E8BFE38F87AA
:10380000988BA98BBA8B26E636E646E655E46F859B
:10381000788989899A890E944039DC01CB018D8B96
:103820009E8BAF8BB88F20E030E040E85FE36D897E
:103830007E898F89988D0E94CA3A88230CF005C032
:1038400081E090E09C8B8B8B1AC020E03FEF4FE72C
:1038500057E46D897E898F89988D0E945E3A18168B
:103860000CF003C01C8A1B8A0AC06D897E898F896F
:10387000988D0E948F37DC01CB019C8B8B8B8B89C1
:103880009C899E878D878D859E850197F1F79E8700
:103890008D8760E070E080E090E00E94803080E002
:1038A00090E0A0E8BFE38B839C83AD83BE8326E6D4
:1038B00036E646E655E46B817C818D819E810E94CF
:1038C0004039DC01CB0189879A87AB87BC8720E030
:1038D00030E040E85FE369857A858B859C850E94AE
:1038E000CA3A88230CF005C081E090E098878F8366
:1038F0001AC020E03FEF4FE757E469857A858B8552
:103900009C850E945E3A18160CF003C018861F8230
:103910000AC069857A858B859C850E948F37DC017A
:10392000CB0198878F838F8198859A83898389813A
:103930009A810197F1F79A8389830E94351EE09658
:103940000FB6F894DEBF0FBECDBFDF91CF910895C3
:10395000CF93DF93CDB7DEB72C970FB6F894DEBFC9
:103960000FBECDBF1092C7021092C60257C080E0B2
:1039700090E0A0E7B1E48B839C83AD83BE8326E611
:1039800036E646E655E46B817C818D819E810E94FE
:103990004039DC01CB0189879A87AB87BC8720E05F
:1039A00030E040E85FE369857A858B859C850E94DD
:1039B000CA3A88230CF005C081E090E098878F8395
:1039C0001AC020E03FEF4FE757E469857A858B8581
:1039D0009C850E945E3A18160CF003C018861F8260
:1039E0000AC069857A858B859C850E948F37DC01AA
:1039F000CB0198878F838F8198859A83898389816A
:103A00009A810197F1F79A8389838091C6029091F8
:103A1000C70201969093C7028093C6028091C602A6
:103A20009091C7028A3091050CF4A1CF2C960FB665
:103A3000F894DEBF0FBECDBFDF91CF910895CF9335
:103A4000DF93CDB7DEB72C970FB6F894DEBF0FBE6D
:103A5000CDBF1092C7021092C60257C080E090E01E
:103A6000A0EAB0E48B839C83AD83BE8326E636E672
:103A700046E655E46B817C818D819E810E944039B0
:103A8000DC01CB0189879A87AB87BC8720E030E0D7
:103A900040E85FE369857A858B859C850E94CA3AF8
:103AA00088230CF005C081E090E098878F831AC0CE
:103AB00020E03FEF4FE757E469857A858B859C8549
:103AC0000E945E3A18160CF003C018861F820AC0C6
:103AD00069857A858B859C850E948F37DC01CB01B7
:103AE00098878F838F8198859A83898389819A812A
:103AF0000197F1F79A8389838091C6029091C7025A
:103B000001969093C7028093C6028091C60290915D
:103B1000C702843691050CF4A1CF2C960FB6F89409
:103B2000DEBF0FBECDBFDF91CF910895CF93DF935E
:103B3000CDB7DEB72C970FB6F894DEBF0FBECDBF62
:103B40001092C7021092C60257C080E090E0A0EA2F
:103B5000B0E48B839C83AD83BE8326E636E646E6DF
:103B600055E46B817C818D819E810E944039DC010E
:103B7000CB0189879A87AB87BC8720E030E040E89B
:103B80005FE369857A858B859C850E94CA3A882384
:103B90000CF005C081E090E098878F831AC020E088
:103BA0003FEF4FE757E469857A858B859C850E94B6
:103BB0005E3A18160CF003C018861F820AC0698589
:103BC0007A858B859C850E948F37DC01CB01988795
:103BD0008F838F8198859A83898389819A810197C0
:103BE000F1F79A8389838091C6029091C70201966A
:103BF0009093C7028093C6028091C6029091C7023B
:103C0000843191050CF4A1CF2C960FB6F894DEBF49
:103C10000FBECDBFDF91CF910895CF93DF93CDB786
:103C2000DEB7E7E2F0E080E68083E6E2F0E087EEF0
:103C30008083DF91CF910895CF93DF93CDB7DEB727
:103C4000EBE2F0E01082EAE2F0E088E08083E5E970
:103C5000F0E086E08083E0E9F0E01082E9E2F0E065
:103C60008FE58083DF91CF9108950F931F93CF93BA
:103C7000DF93CDB7DEB7CC59D0400FB6F894DEBF96
:103C80000FBECDBFFE01ED56FF4F80E090E0A0E8F3
:103C9000BFE380839183A283B3838E0107561F4FB6
:103CA000FE01ED56FF4F26E636E646E655E4608116
:103CB0007181828193810E944039DC01CB01F8013E
:103CC00080839183A283B383FE01E756FF4F20E0F8
:103CD00030E040E85FE360817181828193810E94DE
:103CE000CA3A88230CF008C0FE01E956FF4F81E074
:103CF00090E09183808327C0FE01E756FF4F20E0CC
:103D00003FEF4FE757E460817181828193810E9488
:103D10005E3A18160CF006C0FE01E956FF4F1182FC
:103D2000108211C08E0109561F4FFE01E756FF4F4A
:103D300060817181828193810E948F37DC01CB0188
:103D4000F80191838083DE01AF56BF4FFE01E95633
:103D5000FF4F808191818D939C93FE01EF56FF4F21
:103D6000808191810197F1F7FE01EF56FF4F91831A
:103D7000808380E091E00E945B30FE01E957FF4FB5
:103D800080E090E0A0E8BFE380839183A283B383C7
:103D90008E0103571F4FFE01E957FF4F26E636E617
:103DA00046E655E460817181828193810E944039A9
:103DB000DC01CB01F80180839183A283B383FE01F0
:103DC000E357FF4F20E030E040E85FE3608171811E
:103DD000828193810E94CA3A88230CF008C0FE01B8
:103DE000E557FF4F81E090E09183808327C0FE017B
:103DF000E357FF4F20E03FEF4FE757E460817181C9
:103E0000828193810E945E3A18160CF006C0FE0172
:103E1000E557FF4F1182108211C08E0105571F4FC9
:103E2000FE01E357FF4F60817181828193810E947F
:103E30008F37DC01CB01F80191838083DE01AB5722
:103E4000BF4FFE01E557FF4F808191818D939C9379
:103E5000FE01EB57FF4F808191810197F1F7FE0141
:103E6000EB57FF4F9183808360E070E081E090E04A
:103E70000E948030FE01E558FF4F80E090E0A0E80E
:103E8000BFE380839183A283B3838E010F571F4FBB
:103E9000FE01E558FF4F26E636E646E655E460812A
:103EA0007181828193810E944039DC01CB01F8014C
:103EB00080839183A283B383FE01EF57FF4F20E0FD
:103EC00030E040E85FE360817181828193810E94EC
:103ED000CA3A88230CF008C0FE01E158FF4F81E088
:103EE00090E09183808327C0FE01EF57FF4F20E0D1
:103EF0003FEF4FE757E460817181828193810E9497
:103F00005E3A18160CF006C0FE01E158FF4F118210
:103F1000108211C08E0101581F4FFE01EF57FF4F55
:103F200060817181828193810E948F37DC01CB0196
:103F3000F80191838083DE01A758BF4FFE01E1584D
:103F4000FF4F808191818D939C93FE01E758FF4F35
:103F5000808191810197F1F7FE01E758FF4F91832E
:103F6000808385E191E00E945B30FE01E159FF4FC3
:103F700080E090E0A0E8BFE380839183A283B383D5
:103F80008E010B581F4FFE01E159FF4F26E636E622
:103F900046E655E460817181828193810E944039B7
:103FA000DC01CB01F80180839183A283B383FE01FE
:103FB000EB58FF4F20E030E040E85FE36081718123
:103FC000828193810E94CA3A88230CF008C0FE01C6
:103FD000ED58FF4F81E090E09183808327C0FE0180
:103FE000EB58FF4F20E03FEF4FE757E460817181CE
:103FF000828193810E945E3A18160CF006C0FE0181
:10400000ED58FF4F1182108211C08E010D581F4FC5
:10401000FE01EB58FF4F60817181828193810E9484
:104020008F37DC01CB01F80191838083DE01A35936
:10403000BF4FFE01ED58FF4F808191818D939C937E
:10404000FE01E359FF4F808191810197F1F7FE0155
:10405000E359FF4F918380836AE070E081E090E054
:104060000E948030FE01ED59FF4F80E090E0A0E813
:10407000BFE380839183A283B3838E0107591F4FCF
:10408000FE01ED59FF4F26E636E646E655E460812F
:104090007181828193810E944039DC01CB01F8015A
:1040A00080839183A283B383FE01E759FF4F20E011
:1040B00030E040E85FE360817181828193810E94FA
:1040C000CA3A88230CF008C0FE01E959FF4F81E08D
:1040D00090E09183808327C0FE01E759FF4F20E0E5
:1040E0003FEF4FE757E460817181828193810E94A5
:1040F0005E3A18160CF006C0FE01E959FF4F118216
:10410000108211C08E0109591F4FFE01E759FF4F60
:1041100060817181828193810E948F37DC01CB01A4
:10412000F80191838083DE01AF59BF4FFE01E95949
:10413000FF4F808191818D939C93FE01EF59FF4F3A
:10414000808191810197F1F7FE01EF59FF4F918333
:1041500080838BE191E00E945B30FE01E95AFF4FC2
:1041600080E090E0A0E8BFE380839183A283B383E3
:104170008E01035A1F4FFE01E95AFF4F26E636E62D
:1041800046E655E460817181828193810E944039C5
:10419000DC01CB01F80180839183A283B383FE010C
:1041A000E35AFF4F20E030E040E85FE36081718137
:1041B000828193810E94CA3A88230CF008C0FE01D4
:1041C000E55AFF4F81E090E09183808327C0FE0194
:1041D000E35AFF4F20E03FEF4FE757E460817181E2
:1041E000828193810E945E3A18160CF006C0FE018F
:1041F000E55AFF4F1182108211C08E01055A1F4FE0
:10420000FE01E35AFF4F60817181828193810E9498
:104210008F37DC01CB01F80191838083DE01AB5A3B
:10422000BF4FFE01E55AFF4F808191818D939C9392
:10423000FE01EB5AFF4F808191810197F1F7FE015A
:10424000EB5AFF4F9183808360E070E082E090E062
:104250000E948030FE01E55BFF4F80E090E0A0E827
:10426000BFE380839183A283B3838E010F5A1F4FD4
:10427000FE01E55BFF4F26E636E646E655E4608143
:104280007181828193810E944039DC01CB01F80168
:1042900080839183A283B383FE01EF5AFF4F20E016
:1042A00030E040E85FE360817181828193810E9408
:1042B000CA3A88230CF008C0FE01E15BFF4F81E0A1
:1042C00090E09183808327C0FE01EF5AFF4F20E0EA
:1042D0003FEF4FE757E460817181828193810E94B3
:1042E0005E3A18160CF006C0FE01E15BFF4F11822A
:1042F000108211C08E01015B1F4FFE01EF5AFF4F6C
:1043000060817181828193810E948F37DC01CB01B2
:10431000F80191838083DE01A75BBF4FFE01E15B63
:10432000FF4F808191818D939C93FE01E75BFF4F4E
:10433000808191810197F1F7FE01E75BFF4F918347
:10434000808381E291E00E945B30FE01FF9680E075
:1043500090E0A0E8BFE380839183A283B3838E01C2
:104360000B5B1F4FFE01FF9626E636E646E655E458
:1043700060817181828193810E944039DC01CB018F
:10438000F80180839183A283B383FE01EB5BFF4F2F
:1043900020E030E040E85FE36081718182819381B9
:1043A0000E94CA3A88230CF008C0FE01ED5BFF4F63
:1043B00081E090E09183808327C0FE01EB5BFF4F9B
:1043C00020E03FEF4FE757E4608171818281938164
:1043D0000E945E3A18160CF006C0FE01ED5BFF4F1E
:1043E0001182108211C08E010D5B1F4FFE01EB5B2D
:1043F000FF4F60817181828193810E948F37DC0140
:10440000CB01F80191838083FE01ED5BFF4F80813A
:1044100091819EAF8DAF8DAD9EAD0197F1F79EAFAF
:104420008DAF6AE070E082E090E00E94803080E032
:1044300090E0A0E8BFE38BAB9CABADABBEAB26E698
:1044400036E646E655E46BA97CA98DA99EA90E9493
:104450004039DC01CB0189AF9AAFABAFBCAF20E0F4
:1044600030E040E85FE369AD7AAD8BAD9CAD0E9472
:10447000CA3A88230CF005C081E090E098AF8FAB7A
:104480001AC020E03FEF4FE757E469AD7AAD8BAD3E
:104490009CAD0E945E3A18160CF003C018AE1FAA1D
:1044A0000AC069AD7AAD8BAD9CAD0E948F37DC013F
:1044B000CB0198AF8FAB8FA998AD9AAB89AB89A987
:1044C0009AA90197F1F79AAB89AB87E291E00E9434
:1044D0005B3080E090E0A0E8BFE38FA398A7A9A796
:1044E000BAA726E636E646E655E46FA178A589A583
:1044F0009AA50E944039DC01CB018DA79EA7AFA7EA
:10450000B8AB20E030E040E85FE36DA57EA58FA565
:1045100098A90E94CA3A88230CF005C081E090E077
:104520009CA78BA71AC020E03FEF4FE757E46DA58B
:104530007EA58FA598A90E945E3A18160CF003C0BC
:104540001CA61BA60AC06DA57EA58FA598A90E94D2
:104550008F37DC01CB019CA78BA78BA59CA59EA3C5
:104560008DA38DA19EA10197F1F79EA38DA360E07D
:1045700070E083E090E00E94803080E090E0A0E86E
:10458000BFE38B8F9C8FAD8FBE8F26E636E646E667
:1045900055E46B8D7C8D8D8D9E8D0E944039DC01A4
:1045A000CB0189A39AA3ABA3BCA320E030E040E8F1
:1045B0005FE369A17AA18BA19CA10E94CA3A8823DA
:1045C0000CF005C081E090E098A38F8F1AC020E026
:1045D0003FEF4FE757E469A17AA18BA19CA10E940C
:1045E0005E3A18160CF003C018A21F8E0AC069A10B
:1045F0007AA18BA19CA10E948F37DC01CB0198A3EB
:104600008F8F8F8D98A19A8F898F898D9A8D019721
:10461000F1F79A8F898F8DE291E00E945B3080E004
:1046200090E0A0E8BFE38F87988BA98BBA8B26E632
:1046300036E646E655E46F85788989899A890E942D
:104640004039DC01CB018D8B9E8BAF8BB88F20E086
:1046500030E040E85FE36D897E898F89988D0E9404
:10466000CA3A88230CF005C081E090E09C8B8B8BCC
:104670001AC020E03FEF4FE757E46D897E898F89AC
:10468000988D0E945E3A18160CF003C01C8A1B8A93
:104690000AC06D897E898F89988D0E948F37DC01D1
:1046A000CB019C8B8B8B8B899C899E878D878D857D
:1046B0009E850197F1F79E878D876AE070E083E021
:1046C00090E00E94803080E090E0A0E8BFE38B8320
:1046D0009C83AD83BE8326E636E646E655E46B81D1
:1046E0007C818D819E810E944039DC01CB018987CC
:1046F0009A87AB87BC8720E030E040E85FE36985BC
:104700007A858B859C850E94CA3A88230CF005C067
:1047100081E090E098878F831AC020E03FEF4FE759
:1047200057E469857A858B859C850E945E3A1816C8
:104730000CF003C018861F820AC069857A858B85B4
:104740009C850E948F37DC01CB0198878F838F81F6
:1047500098859A83898389819A810197F1F79A8351
:10476000898383E391E00E945B30C456DF4F0FB62C
:10477000F894DEBF0FBECDBFDF91CF911F910F9197
:1047800008950F931F93CF93DF93CDB7DEB7CC5F20
:10479000D0400FB6F894DEBF0FBECDBFFE01ED5086
:1047A000FF4F80E090E0A0E8BFE380839183A28385
:1047B000B3838E0107501F4FFE01ED50FF4F26E6D9
:1047C00036E646E655E460817181828193810E94DC
:1047D0004039DC01CB01F80180839183A283B3834C
:1047E000FE01E750FF4F20E030E040E85FE36081EA
:1047F0007181828193810E94CA3A88230CF008C09B
:10480000FE01E950FF4F81E090E09183808327C053
:10481000FE01E750FF4F20E03FEF4FE757E4608194
:104820007181828193810E945E3A18160CF006C055
:10483000FE01E950FF4F1182108211C08E01095014
:104840001F4FFE01E750FF4F60817181828193818C
:104850000E948F37DC01CB01F80191838083DE0158
:10486000AF50BF4FFE01E950FF4F808191818D9382
:104870009C93FE01EF50FF4F808191810197F1F7EA
:10488000FE01EF50FF4F9183808363E070E080E092
:1048900090E00E948030FE01E951FF4F80E090E0FF
:1048A000A0E8BFE380839183A283B3838E01035189
:1048B0001F4FFE01E951FF4F26E636E646E655E476
:1048C00060817181828193810E944039DC01CB013A
:1048D000F80180839183A283B383FE01E351FF4FEC
:1048E00020E030E040E85FE3608171818281938164
:1048F0000E94CA3A88230CF008C0FE01E551FF4F20
:1049000081E090E09183808327C0FE01E351FF4F57
:1049100020E03FEF4FE757E460817181828193810E
:104920000E945E3A18160CF006C0FE01E551FF4FDA
:104930001182108211C08E0105511F4FFE01E351FB
:10494000FF4F60817181828193810E948F37DC01EA
:10495000CB01F80191838083DE01AB51BF4FFE0193
:10496000E551FF4F808191818D939C93FE01EB5126
:10497000FF4F808191810197F1F7FE01EB51FF4FCD
:104980009183808383EA91E00E945B30FE01E552CF
:10499000FF4F80E090E0A0E8BFE380839183A28393
:1049A000B3838E010F511F4FFE01E552FF4F26E6E4
:1049B00036E646E655E460817181828193810E94EA
:1049C0004039DC01CB01F80180839183A283B3835A
:1049D000FE01EF51FF4F20E030E040E85FE36081EF
:1049E0007181828193810E94CA3A88230CF008C0A9
:1049F000FE01E152FF4F81E090E09183808327C068
:104A0000FE01EF51FF4F20E03FEF4FE757E4608199
:104A10007181828193810E945E3A18160CF006C063
:104A2000FE01E152FF4F1182108211C08E0101522E
:104A30001F4FFE01EF51FF4F608171818281938191
:104A40000E948F37DC01CB01F80191838083DE0166
:104A5000A752BF4FFE01E152FF4F808191818D939C
:104A60009C93FE01E752FF4F808191810197F1F7FE
:104A7000FE01E752FF4F9183808365E070E081E0A3
:104A800090E00E948030FE01E153FF4F80E090E013
:104A9000A0E8BFE380839183A283B3838E010B528E
:104AA0001F4FFE01E153FF4F26E636E646E655E48A
:104AB00060817181828193810E944039DC01CB0148
:104AC000F80180839183A283B383FE01EB52FF4FF1
:104AD00020E030E040E85FE3608171818281938172
:104AE0000E94CA3A88230CF008C0FE01ED52FF4F25
:104AF00081E090E09183808327C0FE01EB52FF4F5D
:104B000020E03FEF4FE757E460817181828193811C
:104B10000E945E3A18160CF006C0FE01ED52FF4FDF
:104B20001182108211C08E010D521F4FFE01EB52F7
:104B3000FF4F60817181828193810E948F37DC01F8
:104B4000CB01F80191838083DE01A353BF4FFE01A7
:104B5000ED52FF4F808191818D939C93FE01E35331
:104B6000FF4F808191810197F1F7FE01E353FF4FE1
:104B7000918380838FEA91E00E945B30FE01ED53C8
:104B8000FF4F80E090E0A0E8BFE380839183A283A1
:104B9000B3838E0107531F4FFE01ED53FF4F26E6EF
:104BA00036E646E655E460817181828193810E94F8
:104BB0004039DC01CB01F80180839183A283B38368
:104BC000FE01E753FF4F20E030E040E85FE3608103
:104BD0007181828193810E94CA3A88230CF008C0B7
:104BE000FE01E953FF4F81E090E09183808327C06D
:104BF000FE01E753FF4F20E03FEF4FE757E46081AE
:104C00007181828193810E945E3A18160CF006C071
:104C1000FE01E953FF4F1182108211C08E0109532A
:104C20001F4FFE01E753FF4F6081718182819381A5
:104C30000E948F37DC01CB01F80191838083DE0174
:104C4000AF53BF4FFE01E953FF4F808191818D9398
:104C50009C93FE01EF53FF4F808191810197F1F703
:104C6000FE01EF53FF4F9183808366E070E082E0A6
:104C700090E00E948030FE01E954FF4F80E090E018
:104C8000A0E8BFE380839183A283B3838E010354A2
:104C90001F4FFE01E954FF4F26E636E646E655E48F
:104CA00060817181828193810E944039DC01CB0156
:104CB000F80180839183A283B383FE01E354FF4F05
:104CC00020E030E040E85FE3608171818281938180
:104CD0000E94CA3A88230CF008C0FE01E554FF4F39
:104CE00081E090E09183808327C0FE01E354FF4F71
:104CF00020E03FEF4FE757E460817181828193812B
:104D00000E945E3A18160CF006C0FE01E554FF4FF3
:104D10001182108211C08E0105541F4FFE01E35411
:104D2000FF4F60817181828193810E948F37DC0106
:104D3000CB01F80191838083DE01AB54BF4FFE01AC
:104D4000E554FF4F808191818D939C93FE01EB543C
:104D5000FF4F808191810197F1F7FE01EB54FF4FE6
:104D6000918380838FEB91E00E945B300E941F1D36
:104D70000E941F1D66E070E082E090E00E9480309B
:104D8000FE01E555FF4F80E090E0A0E8BFE380839F
:104D90009183A283B3838E010F541F4FFE01E5550B
:104DA000FF4F26E636E646E655E460817181828152
:104DB00093810E944039DC01CB01F801808391830B
:104DC000A283B383FE01EF54FF4F20E030E040E8C0
:104DD0005FE360817181828193810E94CA3A882356
:104DE0000CF008C0FE01E155FF4F81E090E0918397
:104DF000808327C0FE01EF54FF4F20E03FEF4FE7D5
:104E000057E460817181828193810E945E3A181615
:104E10000CF006C0FE01E155FF4F1182108211C057
:104E20008E0101551F4FFE01EF54FF4F60817181CC
:104E3000828193810E948F37DC01CB01F80191833D
:104E40008083DE01A755BF4FFE01E155FF4F8081F2
:104E500091818D939C93FE01E755FF4F8081918155
:104E60000197F1F7FE01E755FF4F918380838DECA9
:104E700091E00E945B300E941F1D0E941F1D66E092
:104E800070E082E090E00E948030FE01E156FF4F2A
:104E900080E090E0A0E8BFE380839183A283B383A6
:104EA0008E010B551F4FFE01E156FF4F26E636E6F9
:104EB00046E655E460817181828193810E94403988
:104EC000DC01CB01F80180839183A283B383FE01CF
:104ED000EB55FF4F20E030E040E85FE360817181F7
:104EE000828193810E94CA3A88230CF008C0FE0197
:104EF000ED55FF4F81E090E09183808327C0FE0154
:104F0000EB55FF4F20E03FEF4FE757E460817181A1
:104F1000828193810E945E3A18160CF006C0FE0151
:104F2000ED55FF4F1182108211C08E010D551F4F9C
:104F3000FE01EB55FF4F60817181828193810E9458
:104F40008F37DC01CB01F80191838083DE01A3560A
:104F5000BF4FFE01ED55FF4F808191818D939C9352
:104F6000FE01E356FF4F808191810197F1F7FE0129
:104F7000E356FF4F918380838BED91E00E945B307D
:104F80000E941F1D0E941F1D66E070E082E090E0FD
:104F90000E948030FE01ED56FF4F80E090E0A0E8D7
:104FA000BFE380839183A283B3838E0107561F4F93
:104FB000FE01ED56FF4F26E636E646E655E46081F3
:104FC0007181828193810E944039DC01CB01F8011B
:104FD00080839183A283B383FE01E756FF4F20E0D5
:104FE00030E040E85FE360817181828193810E94BB
:104FF000CA3A88230CF008C0FE01E956FF4F81E051
:1050000090E09183808327C0FE01E756FF4F20E0A8
:105010003FEF4FE757E460817181828193810E9465
:105020005E3A18160CF006C0FE01E956FF4F1182D9
:10503000108211C08E0109561F4FFE01E756FF4F27
:1050400060817181828193810E948F37DC01CB0165
:10505000F80191838083DE01AF56BF4FFE01E95610
:10506000FF4F808191818D939C93FE01EF56FF4FFE
:10507000808191810197F1F7FE01EF56FF4F9183F7
:10508000808389EE91E00E945B300E941F1D0E9488
:105090001F1D66E070E082E090E00E948030FE011B
:1050A000E957FF4F80E090E0A0E8BFE38083918361
:1050B000A283B3838E0103571F4FFE01E957FF4FB1
:1050C00026E636E646E655E4608171818281938169
:1050D0000E944039DC01CB01F80180839183A283D7
:1050E000B383FE01E357FF4F20E030E040E85FE389
:1050F00060817181828193810E94CA3A88230CF079
:1051000008C0FE01E557FF4F81E090E09183808366
:1051100027C0FE01E357FF4F20E03FEF4FE757E482
:1051200060817181828193810E945E3A18160CF031
:1051300006C0FE01E557FF4F1182108211C08E019B
:1051400005571F4FFE01E357FF4F60817181828138
:1051500093810E948F37DC01CB01F801918380831A
:10516000DE01AB57BF4FFE01E557FF4F80819181B4
:105170008D939C93FE01EB57FF4F808191810197A6
:10518000F1F7FE01EB57FF4F9183808387EF91E0AA
:105190000E945B300E941F1D0E941F1D66E070E090
:1051A00082E090E00E948030FE01E558FF4F80E0F1
:1051B00090E0A0E8BFE380839183A283B3838E0154
:1051C0000F571F4FFE01E558FF4F26E636E646E62D
:1051D00055E460817181828193810E944039DC01B4
:1051E000CB01F80180839183A283B383FE01EF5743
:1051F000FF4F20E030E040E85FE360817181828111
:1052000093810E94CA3A88230CF008C0FE01E1583D
:10521000FF4F81E090E09183808327C0FE01EF572C
:10522000FF4F20E03FEF4FE757E4608171818281BB
:1052300093810E945E3A18160CF006C0FE01E158F8
:10524000FF4F1182108211C08E0101581F4FFE01C5
:10525000EF57FF4F60817181828193810E948F3768
:10526000DC01CB01F80191838083DE01A758BF4F99
:10527000FE01E158FF4F808191818D939C93FE0147
:10528000E758FF4F808191810197F1F7FE01E758C0
:10529000FF4F9183808385E092E00E945B30FE01A6
:1052A000E159FF4F80E090E0A0E8BFE38083918365
:1052B000A283B3838E010B581F4FFE01E159FF4FAC
:1052C00026E636E646E655E4608171818281938167
:1052D0000E944039DC01CB01F80180839183A283D5
:1052E000B383FE01EB58FF4F20E030E040E85FE37E
:1052F00060817181828193810E94CA3A88230CF077
:1053000008C0FE01ED58FF4F81E090E0918380835B
:1053100027C0FE01EB58FF4F20E03FEF4FE757E477
:1053200060817181828193810E945E3A18160CF02F
:1053300006C0FE01ED58FF4F1182108211C08E0190
:105340000D581F4FFE01EB58FF4F60817181828124
:1053500093810E948F37DC01CB01F8019183808318
:10536000DE01A359BF4FFE01ED58FF4F80819181AF
:105370008D939C93FE01E359FF4F808191810197AA
:10538000F1F7FE01E359FF4F9183808364E070E001
:1053900083E090E00E948030FE01ED59FF4F80E0F5
:1053A00090E0A0E8BFE380839183A283B3838E0162
:1053B00007591F4FFE01ED59FF4F26E636E646E638
:1053C00055E460817181828193810E944039DC01C2
:1053D000CB01F80180839183A283B383FE01E75957
:1053E000FF4F20E030E040E85FE36081718182811F
:1053F00093810E94CA3A88230CF008C0FE01E95943
:10540000FF4F81E090E09183808327C0FE01E75940
:10541000FF4F20E03FEF4FE757E4608171818281C9
:1054200093810E945E3A18160CF006C0FE01E959FD
:10543000FF4F1182108211C08E0109591F4FFE01CA
:10544000E759FF4F60817181828193810E948F377C
:10545000DC01CB01F80191838083DE01AF59BF4F9E
:10546000FE01E959FF4F808191818D939C93FE014C
:10547000EF59FF4F808191810197F1F7FE01EF59BC
:10548000FF4F9183808383E192E00E945B30E8E3E9
:10549000F0E080E280830E941F1DE8E3F0E01082CC
:1054A0000E941F1D66E070E082E090E00E94803064
:1054B000FE01E95AFF4F80E090E0A0E8BFE380835F
:1054C0009183A283B3838E01035A1F4FFE01E95AD1
:1054D000FF4F26E636E646E655E46081718182811B
:1054E00093810E944039DC01CB01F80180839183D4
:1054F000A283B383FE01E35AFF4F20E030E040E88F
:105500005FE360817181828193810E94CA3A88231E
:105510000CF008C0FE01E55AFF4F81E090E0918356
:10552000808327C0FE01E35AFF4F20E03FEF4FE7A3
:1055300057E460817181828193810E945E3A1816DE
:105540000CF006C0FE01E55AFF4F1182108211C017
:105550008E01055A1F4FFE01E35AFF4F6081718192
:10556000828193810E948F37DC01CB01F801918306
:105570008083DE01AB5ABF4FFE01E55AFF4F8081A9
:1055800091818D939C93FE01EB5AFF4F8081918115
:105590000197F1F7FE01EB5AFF4F9183808381E27F
:1055A00092E00E945B30E8E3F0E080E280830E94BA
:1055B000A81CE8E3F0E010820E94A81CE8E3F0E0F9
:1055C00080E280830E94A81CE8E3F0E010820E9441
:1055D000A81CE8E3F0E080E280830E94A81CE8E3D6
:1055E000F0E010820E94A81CE8E3F0E080E28083F3
:1055F0000E94961DE8E3F0E0108266E070E082E031
:1056000090E00E948030FE01E55BFF4F80E090E07B
:10561000A0E8BFE380839183A283B3838E010F5AF6
:105620001F4FFE01E55BFF4F26E636E646E655E4F2
:1056300060817181828193810E944039DC01CB01BC
:10564000F80180839183A283B383FE01EF5AFF4F59
:1056500020E030E040E85FE36081718182819381E6
:105660000E94CA3A88230CF008C0FE01E15BFF4F9C
:1056700081E090E09183808327C0FE01EF5AFF4FC5
:1056800020E03FEF4FE757E4608171818281938191
:105690000E945E3A18160CF006C0FE01E15BFF4F57
:1056A0001182108211C08E01015B1F4FFE01EF5A63
:1056B000FF4F60817181828193810E948F37DC016D
:1056C000CB01F80191838083DE01A75BBF4FFE0110
:1056D000E15BFF4F808191818D939C93FE01E75B9D
:1056E000FF4F808191810197F1F7FE01E75BFF4F4A
:1056F000918380838FE292E00E945B30E8E3F0E0E8
:1057000080E280830E94A81CE8E3F0E010820E94FF
:10571000A81CE8E3F0E080E280830E94A81CE8E394
:10572000F0E010820E94A81CE8E3F0E080E28083B1
:105730000E94A81CE8E3F0E010820E94A81CE8E3A5
:10574000F0E080E280830E94961DE8E3F0E01082A2
:1057500066E070E082E090E00E948030FE01FF96FB
:1057600080E090E0A0E8BFE380839183A283B383CD
:105770008E010B5B1F4FFE01FF9626E636E646E6DE
:1057800055E460817181828193810E944039DC01FE
:10579000CB01F80180839183A283B383FE01EB5B8D
:1057A000FF4F20E030E040E85FE36081718182815B
:1057B00093810E94CA3A88230CF008C0FE01ED5B79
:1057C000FF4F81E090E09183808327C0FE01EB5B77
:1057D000FF4F20E03FEF4FE757E460817181828106
:1057E00093810E945E3A18160CF006C0FE01ED5B34
:1057F000FF4F1182108211C08E010D5B1F4FFE0101
:10580000EB5BFF4F60817181828193810E948F37B2
:10581000DC01CB01F80191838083FE01ED5BFF4F3A
:10582000808191819EAF8DAF8DAD9EAD0197F1F7D7
:105830009EAF8DAF8DE392E00E945B30E8E3F0E035
:1058400080E280830E94A81CE8E3F0E010820E94BE
:10585000A81CE8E3F0E080E280830E94A81CE8E353
:10586000F0E010820E94A81CE8E3F0E080E2808370
:105870000E94A81CE8E3F0E010820E94A81CE8E364
:10588000F0E080E280830E94961DE8E3F0E0108261
:1058900066E070E082E090E00E94803080E090E07E
:1058A000A0E8BFE38BAB9CABADABBEAB26E636E668
:1058B00046E655E46BA97CA98DA99EA90E944039B2
:1058C000DC01CB0189AF9AAFABAFBCAF20E030E0D9
:1058D00040E85FE369AD7AAD8BAD9CAD0E94CA3AFA
:1058E00088230CF005C081E090E098AF8FAB1AC020
:1058F00020E03FEF4FE757E469AD7AAD8BAD9CAD4B
:105900000E945E3A18160CF003C018AE1FAA0AC017
:1059100069AD7AAD8BAD9CAD0E948F37DC01CB01B8
:1059200098AF8FAB8FA998AD9AAB89AB89A99AA98B
:105930000197F1F79AAB89AB8BE492E00E945B3060
:10594000E8E3F0E080E280830E94A81CE8E3F0E056
:1059500010820E94A81CE8E3F0E080E280830E94AD
:10596000A81CE8E3F0E010820E94A81CE8E3F0E045
:1059700080E280830E94A81CE8E3F0E010820E948D
:10598000A81CE8E3F0E080E280830E94961DE8E333
:10599000F0E010820E948B2F80E090E0A0E8BFE34F
:1059A0008FA398A7A9A7BAA726E636E646E655E448
:1059B0006FA178A589A59AA50E944039DC01CB0189
:1059C0008DA79EA7AFA7B8AB20E030E040E85FE32B
:1059D0006DA57EA58FA598A90E94CA3A88230CF0D0
:1059E00005C081E090E09CA78BA71AC020E03FEFA4
:1059F0004FE757E46DA57EA58FA598A90E945E3A52
:105A000018160CF003C01CA61BA60AC06DA57EA527
:105A10008FA598A90E948F37DC01CB019CA78BA78B
:105A20008BA59CA59EA38DA38DA19EA10197F1F7A7
:105A30009EA38DA363E070E081E090E00E9480303F
:105A400080E090E0A0E8BFE38B8F9C8FAD8FBE8F8E
:105A500026E636E646E655E46B8D7C8D8D8D9E8D73
:105A60000E944039DC01CB0189A39AA3ABA3BCA35C
:105A700020E030E040E85FE369A17AA18BA19CA11E
:105A80000E94CA3A88230CF005C081E090E098A3F8
:105A90008F8F1AC020E03FEF4FE757E469A17AA14A
:105AA0008BA19CA10E945E3A18160CF003C018A2AC
:105AB0001F8E0AC069A17AA18BA19CA10E948F3779
:105AC000DC01CB0198A38F8F8F8D98A19A8F898F3E
:105AD000898D9A8D0197F1F79A8F898F89E592E0E8
:105AE0000E945B3080E090E0A0E8BFE38F87988B56
:105AF000A98BBA8B26E636E646E655E46F857889AB
:105B000089899A890E944039DC01CB018D8B9E8B5B
:105B1000AF8BB88F20E030E040E85FE36D897E898D
:105B20008F89988D0E94CA3A88230CF005C081E0C5
:105B300090E09C8B8B8B1AC020E03FEF4FE757E43F
:105B40006D897E898F89988D0E945E3A18160CF0B7
:105B500003C01C8A1B8A0AC06D897E898F89988D33
:105B60000E948F37DC01CB019C8B8B8B8B899C89AE
:105B70009E878D878D859E850197F1F79E878D87FE
:105B800065E070E082E090E00E94803080E090E08C
:105B9000A0E8BFE38B839C83AD83BE8326E636E615
:105BA00046E655E46B817C818D819E810E9440395F
:105BB000DC01CB0189879A87AB87BC8720E030E086
:105BC00040E85FE369857A858B859C850E94CA3AA7
:105BD00088230CF005C081E090E098878F831AC07D
:105BE00020E03FEF4FE757E469857A858B859C85F8
:105BF0000E945E3A18160CF003C018861F820AC075
:105C000069857A858B859C850E948F37DC01CB0165
:105C100098878F838F8198859A83898389819A81D8
:105C20000197F1F79A83898384E692E00E945B30C2
:105C30000E941F1D0E941F1DC450DF4F0FB6F89415
:105C4000DEBF0FBECDBFDF91CF911F910F910895A1
:105C5000CF93DF93CDB7DEB7AE970FB6F894DEBF24
:105C60000FBECDBF9EA78DA7EBE3F0E08DA59EA54F
:105C7000959587959595879595958795959587950C
:105C80008064808380E090E0A8E4B2E48CA39DA3CC
:105C9000AEA3BFA322E539E44DE950E46CA17DA198
:105CA0008EA19FA10E944039DC01CB0189A79AA750
:105CB000ABA7BCA720E030E040E85FE369A57AA588
:105CC0008BA59CA50E94CA3A88230CF003C081E0F2
:105CD00088A718C020E030E04FE753E469A57AA513
:105CE0008BA59CA50E945E3A18160CF002C018A65F
:105CF00009C069A57AA58BA59CA50E948F37DC01F8
:105D0000CB0188A788A58BA38BA18A95F1F78BA3DC
:105D1000EBE3F0E08DA59EA59595879595958795E4
:105D20009595879595958795808380E090E0A0E88C
:105D3000BFE3898F9A8FAB8FBC8F26E636E646E6A7
:105D400055E4698D7A8D8B8D9C8D0E944039DC01E4
:105D5000CB018F8F98A3A9A3BAA320E030E040E83D
:105D60005FE36F8D78A189A19AA10E94CA3A882326
:105D70000CF005C081E090E09E8F8D8F1AC020E06E
:105D80003FEF4FE757E46F8D78A189A19AA10E9458
:105D90005E3A18160CF003C01E8E1D8E0AC06F8D61
:105DA00078A189A19AA10E948F37DC01CB019E8F37
:105DB0008D8F8D8D9E8D988F8F8B8F89988D01976C
:105DC000F1F7988F8F8BEBE3F0E08DA58F708064F7
:105DD000808380E090E0A8E4B2E48E879F87A88B60
:105DE000B98B22E539E44DE950E46E857F858889D9
:105DF00099890E944039DC01CB018B8B9C8BAD8B48
:105E0000BE8B20E030E040E85FE36B897C898D89C0
:105E10009E890E94CA3A88230CF003C081E08A8BD5
:105E200018C020E030E04FE753E46B897C898D890E
:105E30009E890E945E3A18160CF002C01A8A09C0A8
:105E40006B897C898D899E890E948F37DC01CB010B
:105E50008A8B8A898D878D858A95F1F78D87EBE30B
:105E6000F0E08DA58F70808380E090E0A0EAB0E440
:105E70008B839C83AD83BE8326E636E646E655E4F7
:105E80006B817C818D819E810E944039DC01CB0138
:105E900089879A87AB87BC8720E030E040E85FE3E2
:105EA00069857A858B859C850E94CA3A88230CF087
:105EB00005C081E090E098878F831AC020E03FEF13
:105EC0004FE757E469857A858B859C850E945E3A09
:105ED00018160CF003C018861F820AC069857A85DF
:105EE0008B859C850E948F37DC01CB0198878F833F
:105EF0008F8198859A83898389819A810197F1F7A7
:105F00009A838983AE960FB6F894DEBF0FBECDBFDD
:105F1000DF91CF910895CF93DF93CDB7DEB781E0C6
:105F200090E00E94282E1092C5021092C402DF91C8
:105F3000CF910895CF93DF93CDB7DEB768970FB6B3
:105F4000F894DEBF0FBECDBF80E090E0A0E7B1E4E3
:105F50008F87988BA98BBA8B26E636E646E655E402
:105F60006F85788989899A890E944039DC01CB0143
:105F70008D8B9E8BAF8BB88F20E030E040E85FE3E5
:105F80006D897E898F89988D0E94CA3A88230CF08A
:105F900005C081E090E09C8B8B8B1AC020E03FEF26
:105FA0004FE757E46D897E898F89988D0E945E3A0C
:105FB00018160CF003C01C8A1B8A0AC06D897E89E2
:105FC0008F89988D0E948F37DC01CB019C8B8B8B46
:105FD0008B899C899E878D878D859E850197F1F79A
:105FE0009E878D8783E390E00E94282E80E090E0DA
:105FF000A0E8BFE38B839C83AD83BE8326E636E6B1
:1060000046E655E46B817C818D819E810E944039FA
:10601000DC01CB0189879A87AB87BC8720E030E021
:1060200040E85FE369857A858B859C850E94CA3A42
:1060300088230CF005C081E090E098878F831AC018
:1060400020E03FEF4FE757E469857A858B859C8593
:106050000E945E3A18160CF003C018861F820AC010
:1060600069857A858B859C850E948F37DC01CB0101
:1060700098878F838F8198859A83898389819A8174
:106080000197F1F79A83898382E390E00E94282E9A
:1060900088E290E00E94282E8CE090E00E94282E5A
:1060A0000E948B2F68960FB6F894DEBF0FBECDBF4F
:1060B000DF91CF910895CF93DF93CDB7DEB72297CD
:1060C0000FB6F894DEBF0FBECDBF9A8389830AC096
:1060D000E981FA8180810E94073189819A81019644
:1060E0009A838983E981FA818081882389F72296BE
:1060F0000FB6F894DEBF0FBECDBFDF91CF910895EC
:10610000CF93DF93CDB7DEB724970FB6F894DEBFF9
:106110000FBECDBF9A8389837C836B8389819A81EB
:106120009C01220F331F220F331FC901880F991FB3
:10613000880F991F280F391F8B819C81820F931F15
:106140009093C5028093C4028091C4029091C502CD
:10615000843191053CF48091C4029091C50280681D
:106160000E94282E8091C4029091C502843191052D
:10617000ACF08091C4029091C5028832910574F40C
:106180008091C4029091C50224E130E0B9010E94DF
:10619000C040805C9F4F80680E94282E8091C4027E
:1061A0009091C50288329105A4F08091C40290912B
:1061B000C5028C3391056CF48091C4029091C502A4
:1061C00028E230E0B9010E94C040449680680E94F5
:1061D000282E8091C4029091C5028D33910574F0F0
:1061E0008091C4029091C5022CE330E0B9010E9475
:1061F000C0408C5A9F4F80680E94282E24960FB66C
:10620000F894DEBF0FBECDBFDF91CF910895CF933D
:10621000DF93CDB7DEB7A9970FB6F894DEBF0FBEF8
:10622000CDBF89A78091C4029091C50284319105A8
:1062300021F480EC90E00E94282E8091C40290917D
:10624000C5028832910521F484E990E00E94282E4D
:106250008091C4029091C5028C33910521F484EDA4
:1062600090E00E94282EEBE3F0E089A585958595C6
:10627000859585958065808380E090E0A8E4B2E410
:1062800088A399A3AAA3BBA322E539E44DE950E46E
:1062900068A179A18AA19BA10E944039DC01CB01B0
:1062A0008DA39EA3AFA3B8A720E030E040E85FE352
:1062B0006DA17EA18FA198A50E94CA3A88230CF0F7
:1062C00003C081E08CA318C020E030E04FE753E426
:1062D0006DA17EA18FA198A50E945E3A18160CF0C0
:1062E00002C01CA209C06DA17EA18FA198A50E9429
:1062F0008F37DC01CB018CA38CA18F8F8F8D8A957A
:10630000F1F78F8FEBE3F0E089A58595859585956D
:1063100085958061808380E090E0A8E4B2E48E8B74
:106320009F8BA88FB98F22E539E44DE950E46E893F
:106330007F89888D998D0E944039DC01CB018B8F3C
:106340009C8FAD8FBE8F20E030E040E85FE36B8D27
:106350007C8D8D8D9E8D0E94CA3A88230CF003C0DF
:1063600081E08A8F18C020E030E04FE753E46B8D66
:106370007C8D8D8D9E8D0E945E3A18160CF002C0A9
:106380001A8E09C06B8D7C8D8D8D9E8D0E948F37EE
:10639000DC01CB018A8F8A8D8D8B8D898A95F1F7EF
:1063A0008D8BEBE3F0E089A58F708065808380E0C2
:1063B00090E0A8E4B2E48C879D87AE87BF8722E592
:1063C00039E44DE950E46C857D858E859F850E947A
:1063D0004039DC01CB01898B9A8BAB8BBC8B20E0E5
:1063E00030E040E85FE369897A898B899C890E9463
:1063F000CA3A88230CF003C081E0888B18C020E0E3
:1064000030E04FE753E469897A898B899C890E943F
:106410005E3A18160CF002C0188A09C069897A8998
:106420008B899C890E948F37DC01CB01888B8889FE
:106430008B878B858A95F1F78B87EBE3F0E089A555
:106440008F708061808380E090E0A8E4B2E48A836A
:106450009B83AC83BD8322E539E44DE950E46A8136
:106460007B818C819D810E944039DC01CB018F832F
:106470009887A987BA8720E030E040E85FE36F8122
:10648000788589859A850E94CA3A88230CF003C0D2
:1064900081E08E8318C020E030E04FE753E46F8145
:1064A000788589859A850E945E3A18160CF002C09C
:1064B0001E8209C06F81788589859A850E948F37F1
:1064C000DC01CB018E838E81898389818A95F1F7E6
:1064D00089838091C4029091C50201969093C50270
:1064E0008093C4028091C4029091C50280359105C9
:1064F00021F41092C5021092C402A9960FB6F89426
:10650000DEBF0FBECDBFDF91CF910895CF93DF9354
:10651000CDB7DEB7E0970FB6F894DEBF0FBECDBFA4
:10652000E8E3F0E081E0808380E090E0A0EAB0E47E
:106530008FA398A7A9A7BAA726E636E646E655E4AC
:106540006FA178A589A59AA50E944039DC01CB01ED
:106550008DA79EA7AFA7B8AB20E030E040E85FE38F
:106560006DA57EA58FA598A90E94CA3A88230CF034
:1065700005C081E090E09CA78BA71AC020E03FEF08
:106580004FE757E46DA57EA58FA598A90E945E3AB6
:1065900018160CF003C01CA61BA60AC06DA57EA58C
:1065A0008FA598A90E948F37DC01CB019CA78BA7F0
:1065B0008BA59CA59EA38DA38DA19EA10197F1F70C
:1065C0009EA38DA3EBE2F0E080819927807290700A
:1065D0000097C1F3ECE2F0E080E88083EBE2F0E0CA
:1065E00080819927807290700097C1F3ECE2F0E00F
:1065F00082E08083EBE2F0E08081992780729070E6
:106600000097C1F3ECE2F0E01082EBE2F0E0808171
:106610009927807290700097C1F380E090E0A0EA23
:10662000B0E48B8F9C8FAD8FBE8F26E636E646E6B4
:1066300055E46B8D7C8D8D8D9E8D0E944039DC01E3
:10664000CB0189A39AA3ABA3BCA320E030E040E830
:106650005FE369A17AA18BA19CA10E94CA3A882319
:106660000CF005C081E090E098A38F8F1AC020E065
:106670003FEF4FE757E469A17AA18BA19CA10E944B
:106680005E3A18160CF003C018A21F8E0AC069A14A
:106690007AA18BA19CA10E948F37DC01CB0198A32A
:1066A0008F8F8F8D98A19A8F898F898D9A8D019761
:1066B000F1F79A8F898FE8E3F0E0108280E090E0B4
:1066C000A0EAB0E48F87988BA98BBA8B26E636E6D2
:1066D00046E655E46F85788989899A890E94403910
:1066E000DC01CB018D8B9E8BAF8BB88F20E030E02F
:1066F00040E85FE36D897E898F89988D0E94CA3A50
:1067000088230CF005C081E090E09C8B8B8B1AC035
:1067100020E03FEF4FE757E46D897E898F89988DA0
:106720000E945E3A18160CF003C01C8A1B8A0AC02D
:106730006D897E898F89988D0E948F37DC01CB010E
:106740009C8B8B8B8B899C899E878D878D859E8565
:106750000197F1F79E878D87E8E3F0E081E0808381
:1067600080E090E0A0EAB0E48B839C83AD83BE839D
:1067700026E636E646E655E46B817C818D819E8176
:106780000E944039DC01CB0189879A87AB87BC879F
:1067900020E030E040E85FE369857A858B859C8561
:1067A0000E94CA3A88230CF005C081E090E09887E7
:1067B0008F831AC020E03FEF4FE757E469857A8561
:1067C0008B859C850E945E3A18160CF003C01886D3
:1067D0001F820AC069857A858B859C850E948F37C8
:1067E000DC01CB0198878F838F8198859A83898379
:1067F00089819A810197F1F79A838983E0960FB690
:10680000F894DEBF0FBECDBFDF91CF910895CF9337
:10681000DF93CDB7DEB724970FB6F894DEBF0FBE77
:10682000CDBF9A8389837C836B83EBE2F0E0808128
:106830009927807290700097C1F3ECE2F0E080E855
:106840008083EBE2F0E0808199278072907000975E
:10685000C1F3ECE2F0E01082EBE2F0E080819927F6
:10686000807290700097C1F3ECE2F0E081E08083E9
:10687000EBE2F0E080819927807290700097C1F37D
:10688000ECE2F0E089818083EBE2F0E080819927FF
:10689000807290700097C1F3EBE2F0E0808199275D
:1068A000807290700097C1F3ECE2F0E080E88083A2
:1068B000EBE2F0E080819927807290700097C1F33D
:1068C000ECE2F0E01082EBE2F0E080819927807248
:1068D00090700097C1F3ECE2F0E082E08083EBE29D
:1068E000F0E080819927807290700097C1F3ECE20C
:1068F000F0E08B818083EBE2F0E080819927807269
:1069000090700097C1F324960FB6F894DEBF0FBEC7
:10691000CDBFDF91CF910895CF93DF93CDB7DEB791
:1069200024970FB6F894DEBF0FBECDBF9A8389833C
:106930007C836B83EBE2F0E080819927807290701A
:106940000097C1F3ECE2F0E080E88083EBE2F0E056
:1069500080819927807290700097C1F3ECE2F0E09B
:106960001082EBE2F0E080819927807290700097AE
:10697000C1F3ECE2F0E01082EBE2F0E080819927D5
:10698000807290700097C1F3ECE2F0E0898180831F
:10699000EBE2F0E080819927807290700097C1F35C
:1069A000EBE2F0E080819927807290700097C1F34C
:1069B000ECE2F0E080E88083EBE2F0E08081992770
:1069C000807290700097C1F3ECE2F0E01082EBE28D
:1069D000F0E080819927807290700097C1F3ECE21B
:1069E000F0E083E08083EBE2F0E080819927807221
:1069F00090700097C1F3ECE2F0E08B818083EBE2D2
:106A0000F0E080819927807290700097C1F32496FE
:106A10000FB6F894DEBF0FBECDBFDF91CF910895C2
:106A2000CF93DF93CDB7DEB722970FB6F894DEBFD2
:106A30000FBECDBF9A838983EBE2F0E08081992776
:106A4000807290700097C1F3ECE2F0E080E8808300
:106A5000EBE2F0E080819927807290700097C1F39B
:106A6000ECE2F0E01082EBE2F0E0808199278072A6
:106A700090700097C1F3ECE2F0E081E08083EBE2FC
:106A8000F0E080819927807290700097C1F3ECE26A
:106A9000F0E089818083EBE2F0E0808199278072C9
:106AA00090700097C1F3EBE2F0E08081992780724B
:106AB00090700097C1F3ECE2F0E080E88083EBE2B5
:106AC000F0E080819927807290700097C1F3ECE22A
:106AD000F0E01082EBE2F0E0808199278072907004
:106AE0000097C1F3ECE2F0E083E08083EBE2F0E0BA
:106AF00080819927807290700097C1F3ECE2F0E0FA
:106B00001082EBE2F0E0808199278072907000970C
:106B1000C1F322960FB6F894DEBF0FBECDBFDF9152
:106B2000CF910895CF93DF93CDB7DEB722970FB6FD
:106B3000F894DEBF0FBECDBF9A838983EBE2F0E00D
:106B400080819927807290700097C1F3ECE2F0E0A9
:106B500080E88083EBE2F0E080819927807290707A
:106B60000097C1F3ECE2F0E01082EBE2F0E080810C
:106B70009927807290700097C1F3ECE2F0E081E019
:106B80008083EBE2F0E0808199278072907000971B
:106B9000C1F3ECE2F0E01082EBE2F0E080819927B3
:106BA000807290700097C1F3EBE2F0E0808199274A
:106BB000807290700097C1F3ECE2F0E080E880838F
:106BC000EBE2F0E080819927807290700097C1F32A
:106BD000ECE2F0E01082EBE2F0E080819927807235
:106BE00090700097C1F3ECE2F0E083E08083EBE289
:106BF000F0E080819927807290700097C1F3ECE2F9
:106C0000F0E089818083EBE2F0E080819927807257
:106C100090700097C1F322960FB6F894DEBF0FBEB6
:106C2000CDBFDF91CF910895CF93DF93CDB7DEB77E
:106C3000EBE2F0E080819927807290700097C1F3B9
:106C4000ECE2F0E080E88083EBE2F0E080819927DD
:106C5000807290700097C1F3ECE2F0E01082EBE2FA
:106C6000F0E080819927807290700097C1F3ECE288
:106C7000F0E083E08083EBE2F0E08081992780728E
:106C800090700097C1F3ECE2F0E01082EBE2F0E0EC
:106C900080819927807290700097C1F3DF91CF9126
:106CA0000895CF93DF93CDB7DEB7EBE2F0E08081BC
:106CB0009927807290700097C1F3ECE2F0E080E8D1
:106CC0008083EBE2F0E080819927807290700097DA
:106CD000C1F3ECE2F0E01082EBE2F0E08081992772
:106CE000807290700097C1F3ECE2F0E081E0808365
:106CF000EBE2F0E080819927807290700097C1F3F9
:106D0000ECE2F0E01082EBE2F0E080819927807203
:106D100090700097C1F3DF91CF910895CF93DF93E7
:106D2000CDB7DEB724970FB6F894DEBF0FBECDBF48
:106D30009A8389837C836B83EBE2F0E080819927DF
:106D4000807290700097C1F3ECE2F0E080E88083FD
:106D5000EBE2F0E080819927807290700097C1F398
:106D6000ECE2F0E01082EBE2F0E0808199278072A3
:106D700090700097C1F3ECE2F0E081E08083EBE2F9
:106D8000F0E080819927807290700097C1F3ECE267
:106D9000F0E089818083EBE2F0E0808199278072C6
:106DA00090700097C1F3EBE2F0E080819927807248
:106DB00090700097C1F3ECE2F0E080E88083EBE2B2
:106DC000F0E080819927807290700097C1F3ECE227
:106DD000F0E01082EBE2F0E0808199278072907001
:106DE0000097C1F3ECE2F0E083E08083EBE2F0E0B7
:106DF00080819927807290700097C1F3ECE2F0E0F7
:106E00008B818083EBE2F0E0808199278072907023
:106E10000097C1F324960FB6F894DEBF0FBECDBF26
:106E2000DF91CF910895CF93DF93CDB7DEB724974D
:106E30000FB6F894DEBF0FBECDBF9A8389837C83E3
:106E40006B83EBE2F0E0808199278072907000976D
:106E5000C1F3ECE2F0E080E88083EBE2F0E08081D7
:106E60009927807290700097C1F3ECE2F0E01082F5
:106E7000EBE2F0E080819927807290700097C1F377
:106E8000ECE2F0E01082EBE2F0E080819927807282
:106E900090700097C1F3ECE2F0E089818083EBE22F
:106EA000F0E080819927807290700097C1F3EBE247
:106EB000F0E080819927807290700097C1F3ECE236
:106EC000F0E080E88083EBE2F0E080819927807237
:106ED00090700097C1F3ECE2F0E01082EBE2F0E09A
:106EE00080819927807290700097C1F3ECE2F0E006
:106EF00082E08083EBE2F0E08081992780729070DD
:106F00000097C1F3ECE2F0E08B81808324960FB60A
:106F1000F894DEBF0FBECDBFDF91CF910895EF9201
:106F2000FF920F931F937B018C0120E030E040E043
:106F30005FE40E94943A88237CF020E030E040E057
:106F40005FE4C801B7010E94E2380E94003B605034
:106F500070408040904804C0C801B7010E94003BC7
:106F60001F910F91FF90EF900895A0E0B0E0EBEB40
:106F7000F7E30C94EB40FC016A019081923008F435
:106F80001BC1DB018C91823080F0943061F484303D
:106F900009F012C19181EB018981981709F40CC1A4
:106FA000ECE6F2E009C1843011F4FB0105C1823046
:106FB00091F4923009F000C1EA01DF0188E00D9000
:106FC00009928150E1F78181FB0191818923E601DA
:106FD0008983F601F1C0923041F362807380EB0146
:106FE0008A809B80E480F580068117812C813D8119
:106FF0004E815F815301A818B908C501B7FCABC029
:1070000080970CF457C0861497040CF4BEC034016A
:10701000EE24FF2487019181FB018181981709F4F7
:10702000A6C0992309F49CC02E193F09400B510BAF
:1070300057FDB0C0E60119827B826A82F601248383
:10704000358346835783E6012C813D814E815F81E4
:1070500079018A01DA01C9010197A109B1098F5F9C
:107060009F4FAF4FBF43F8F4E6016A817B81A801CF
:107070009701220F331F441F551F61507040790143
:107080008A01DA01C9010197A109B1098F5F9F4FF8
:10709000AF4FBF4360F3E6017B836A83F60124832D
:1070A00035834683578383E0D6018C9357FD39C0DF
:1070B000F60182C086149704B4F4C0E0D0E0DA018F
:1070C000C90181709070A070B07056954795379542
:1070D0002795282B392B4A2B5B2B2196AC16BD0606
:1070E00071F78A0C9B1C681479040CF094CFC0E0F3
:1070F000D0E05401A618B708D801C701817090707C
:10710000A070B07016950795F794E794E82AF92ACD
:107110000A2B1B2B2196AC16BD0671F76A0C7B1C43
:107120007ACFDA01C901B695A79597958795217011
:10713000307040705070282B392B4A2B5B2BE601A6
:107140002C833D834E835F838A819B8101969B8341
:107150008A83F60131C0882799278A199B0950CF65
:10716000E21AF30A040B150BA801970161CFE6019F
:1071700099837B826A822E0D3F1D401F511FF601AD
:1071800024833583468357838ECF20E030E040E070
:1071900050E041CF81E0E60189837B826A8250958D
:1071A0004095309521953F4F4F4F5F4FF601248317
:1071B00035834683578347CFCF01EEE0CDB7DEB7A7
:1071C0000C940741A0E2B0E0E8EEF8E30C94F34041
:1071D00069837A838B839C832D833E834F83588777
:1071E00089E1E82EF12CEC0EFD1EB701CE010196CF
:1071F0000E94723C8E010F5E1F4FB801CE010596B2
:107200000E94723C8A8991E089278A8BAE01475F90
:107210005F4FB801C7010E94B5370E94503BE6E0BE
:10722000A0960C940F41A0E2B0E0E9E1F9E30C94E0
:10723000F34069837A838B839C832D833E834F83C2
:10724000588799E1E92EF12CEC0EFD1EB701CE0115
:1072500001960E94723C8E010F5E1F4FB801CE0155
:1072600005960E94723CAE01475F5F4FB801C701AF
:107270000E94B5370E94503BE6E0A0960C940F4167
:10728000A0E2B0E0E6E4F9E30C94E74069837A8396
:107290008B839C832D833E834F8358878E01075EAB
:1072A0001F4FB801CE0101960E94723CF1E1EF2E12
:1072B000F12CEC0EFD1EB701CE0105960E94723C2A
:1072C000898D823078F09989923040F420E09A8D4F
:1072D0008A89981321E02A8BB701E9C0843051F4E0
:1072E000923061F020E09A8D8A89981321E02A8FEC
:1072F000B801DDC0943029F4823041F76CE672E0C9
:10730000D6C0823079F3923009F32D8D3E8D4F8DAA
:1073100058A18D899E89AF89B88D222433242101FB
:10732000AA24BB246501EE24FF24870160E070E0FD
:107330000DC06F5F7F4F6032710599F1880F991F03
:10734000AA1FBB1F569547953795279520FF19C053
:10735000280E391E4A1E5B1E662477244301281618
:1073600039064A065B0628F4E1E06E2E712C812C6A
:10737000912CAE0CBF1CC01ED11EA60CB71CC81C85
:10738000D91CEE0CFF1C001F111FB7FFD2CFE1E08C
:107390006E2E712C812C912CE628F72808291929AA
:1073A000C8CF8B8D9C8D2B893C89820F931F0296B1
:1073B0009C878B871A869A8D8A89981711F081E0AD
:1073C0008A87D7FE17C08B859C85A0FE0CC056947B
:1073D00047943794279420E030E040E050E8222A98
:1073E000332A442A552AD694C794B794A794019671
:1073F0009C878B8730E0A31630E0B30630E0C306ED
:1074000030E4D30618F58B859C850EC0220C331C06
:10741000441C551C019720E0A21620E0B20620E093
:10742000C20620E4D20680F4AA0CBB1CCC1CDD1CD6
:1074300057FEECCF31E0632E712C812C912CA628C5
:10744000B728C828D928E2CF9C878B87D601C501E9
:107450008F779070A070B07080349105A105B10550
:1074600051F0AD86BE86CF86D88A83E08987BE017B
:10747000675F7F4F1CC0A7FCF4CF21143104410487
:10748000510479F380E490E0A0E0B0E0A80EB91ECA
:10749000CA1EDB1E80E8682E8FEF782E8FEF882EB5
:1074A0008FEF982EA620B720C820D920DACFCB01A5
:1074B0000E94503BE2E1A0960C940341A8E1B0E0A9
:1074C000E4E6FAE30C94F34069837A838B839C832C
:1074D0002D833E834F83588781E1E82EF12CEC0EFB
:1074E000FD1EB701CE0101960E94723C8E01075F1E
:1074F0001F4FB801CE0105960E94723C89898230E7
:1075000018F42FEF3FEF0BC089858230D0F3B8011C
:10751000C7010E94113D282F332727FD3095C9014F
:10752000E6E068960C940F41A8E1B0E0EAE9FAE3DE
:107530000C94F34069837A838B839C832D833E83F1
:107540004F83588781E1E82EF12CEC0EFD1EB70128
:10755000CE0101960E94723C8E01075F1F4FB80159
:10756000CE0105960E94723C8989823018F42FEF73
:107570003FEF0BC089858230D0F3B801C7010E946C
:10758000113D282F332727FD3095C901E6E0689685
:107590000C940F41A8E1B0E0E0EDFAE30C94F34065
:1075A00069837A838B839C832D833E834F835887A3
:1075B00081E1E82EF12CEC0EFD1EB701CE01019603
:1075C0000E94723C8E01075F1F4FB801CE010596E5
:1075D0000E94723C8989823018F08985823018F4C3
:1075E00021E030E008C0B801C7010E94113D282FFA
:1075F000332727FD3095C901E6E068960C940F41CA
:10760000ACE0B0E0E6E0FBE30C94F74069837A83FA
:107610008B839C83BE016B5F7F4FCE0101960E94DE
:10762000723C8D81823061F0823050F0843069F498
:107630008E81882359F52FEF3FEF4FEF5FE72AC088
:1076400020E030E040E050E025C02F81388537FD54
:10765000F7CF2F31310564F78EE190E0821B930B59
:1076600029853A854B855C8504C0569547953795A5
:1076700027958A95D2F78E81882361F050954095A1
:10768000309521953F4F4F4F5F4F04C020E030E0D1
:1076900040E050E8CA01B901E2E02C960C94134195
:1076A0004F925F926F927F928F929F92AF92BF9212
:1076B000DF92EF92FF920F931F9320E030E040E0C3
:1076C00050E0FC01E480F58006811781D180808143
:1076D000823038F4D801C701A061AF77B0706FEF86
:1076E000D9C0843009F46EC0823009F471C0E1144D
:1076F000F1040105110509F46BC0828193816FEFDC
:10770000823896070CF06AC062E87FEF681B790B3D
:107710006A3171050CF080C047015801062E04C083
:10772000B694A794979487940A94D2F74424552446
:10773000320181E090E0A0E0B0E004C0880F991F22
:10774000AA1FBB1F6A95D2F70197A109B109E822C8
:10775000F9220A231B23E114F1040105110529F084
:1077600061E0462E512C612C712C85017401E428B6
:10777000F52806291729D801C7018F779070A070C6
:10778000B07080349105A105B10509F457C0D80146
:10779000C701CF96A11DB11D60E070E08030E0E030
:1077A0009E07E0E0AE07E0E4BE0710F061E070E0A5
:1077B00027E0B695A795979587952A95D1F7AF7746
:1077C000B07068C080E090E0A0E0B0E06FEF62C011
:1077D00080E090E0A0E0B0E060E05CC0803891051F
:1077E0008CF7BC0161587F4FD801C7018F7790702B
:1077F000A070B07080349105A105B105A1F08FE3B0
:1078000090E0A0E0B0E0E80EF91E0A1F1B1F17FD74
:1078100028C0D801C701CCCF60E070E080E090E0E4
:10782000A0E0B0E0CCCFE7FEF2CF80E490E0A0E0B3
:10783000B0E0E80EF91E0A1F1B1FE9CFE7FC18C0D5
:1078400080E090E060E0E61660E0F60660E00607A3
:1078500060E4160710F081E090E0BC01D801C70198
:10786000A7CF16950795F794E7946F5F7F4FD1CF19
:10787000D801C701805C9F4FAF4FBF4F60E070E001
:107880008030E0E09E07E0E0AE07E0E4BE0708F4E9
:107890008FCF8CCF282F392F9A2F9F77842F8078E6
:1078A000892B962F9795992797958F77482F492B56
:1078B0006695852F8078862BD794DD24D7948F7793
:1078C000582F5D29CA01B9011F910F91FF90EF90C8
:1078D000DF90BF90AF909F908F907F906F905F9060
:1078E0004F900895FC01DB01208131819281492F65
:1078F0004F7750E0991F9927991F8381682F660F52
:10790000692B881F8827881FFD018183662309F062
:1079100049C0211531054105510509F470C082E8BF
:107920009FEFFD0193838283220F331F441F551F56
:10793000220F331F441F551F220F331F441F551F93
:10794000220F331F441F551F220F331F441F551F83
:10795000220F331F441F551F220F331F441F551F73
:1079600083E08C932030F0E03F07F0E04F07F0E435
:107970005F0790F482E89FEF220F331F441F551FCB
:107980000197203060E0360760E0460760E4560764
:1079900098F3FD0193838283FD012483358346831D
:1079A000578308956F3F71F1862F99278F57904025
:1079B000FD019383828383E08C93220F331F441F46
:1079C000551F220F331F441F551F220F331F441F03
:1079D000551F220F331F441F551F220F331F441FF3
:1079E000551F220F331F441F551F220F331F441FE3
:1079F000551F50642483358346835783089582E05E
:107A00008C930895211531054105510519F484E041
:107A10008C93089544FD02C01C92BECF81E08C93EC
:107A2000BBCFEF92FF920F931F93CF93DF93FC0195
:107A3000DB018081823050F09C91923038F08430AC
:107A400041F49430B1F08181882381F461E070E0E9
:107A50004BC09430E9F18230A1F09230A1F3618102
:107A6000ED018981681791F0662381F36FEF7FEF55
:107A70003BC0EB018981682F77278181681B7109E1
:107A800033C0923059F560E070E02EC0228133811E
:107A9000ED018A819B818217930734F328173907F8
:107AA0009CF0E480F58006811781FD0124813581F9
:107AB000468157812E153F0540075107A8F2E2166F
:107AC000F30604071507F8F6662309F0BFCFCECFFB
:107AD000FB018181882309F0B9CFC8CFEB018981EF
:107AE000882309F0B3CFC2CFCB01E6E0CDB7DEB734
:107AF0000C940F410F931F93CF93DF93CDB7DEB755
:107B000060970FB6F894DEBF0FBECDBF0F89188DFA
:107B100086E08E831C830B838FEF9FE798878F838C
:107B2000AE01455E5F4F5A834983698D7A8DCE01E0
:107B300003960E94AC3D29853A85020F131FF80178
:107B4000108260960FB6F894DEBF0FBECDBFDF91F6
:107B5000CF911F910F9108952F923F924F925F9274
:107B60006F927F928F929F92AF92BF92CF92DF924D
:107B7000EF92FF920F931F93CF93DF93CDB7DEB7B2
:107B800064970FB6F894DEBF0FBECDBFCC24DD24C2
:107B900076011C017C8B6B8B2A01FC0117821682FB
:107BA000838181FD03C08FEF9FEF85C2AA24BB2490
:107BB0006FC2A0FE54C28A8980538A30E8F4FA89E1
:107BC000F03341F42D85222329F4A3FC03C080E087
:107BD00091E06FC08AE0ED85E802C0011124FA89C6
:107BE000F80FF053FD87F7FF02C02FE72D87A3FCA6
:107BF00049C23D853E8746C2C50188709070A3FE8C
:107C000005C0ED85EE2311F4F1E0FD872A892836C1
:107C100024F525360CF05BC0233509F480C02435EB
:107C20008CF42B32C1F12C3234F42032C1F12332E6
:107C300009F00AC23CC03A893D32B1F13E3209F046
:107C400003C23AC08A89833609F449C084360CF0ED
:107C500081C0883509F0F8C11BC0EA89E03709F412
:107C6000A3C0E13744F4EC3669F1EF3671F0E93640
:107C700009F0EAC16FC0FA89F53709F49DC0F837F9
:107C800039F0F33709F0E0C134C028E0298B94C003
:107C900030E1398B91C080E190E0A82AB92AE0E276
:107CA000F0E0AE2ABF2AEEC120E830E00DC080E44B
:107CB00090E0A82AB92AE6C1E8E0F0E0AE2ABF2A9F
:107CC0001D86E0C124E030E0A22AB32ADBC13FE3F5
:107CD000C32E3E8531503E8783E68A8B41C1F20137
:107CE000C080FE85F150FE8722E030E0420E531E38
:107CF00037C1F201C080D180892B49F0FD856F2FFB
:107D0000772767FD7095C6010E94884019C0F6016B
:107D100001900020E9F73197EC19E98B12C0F201CC
:107D2000C080D180892B49F0FD856F2F772767FDB3
:107D30007095C6010E947D4003C0C6010E94744038
:107D4000898B22E030E0420E531E3E858989381B24
:107D50003E8706C1A2FE08C0F20180819181A28106
:107D6000B38124E030E009C0F20180819181AA272B
:107D700097FDA095BA2F22E030E0420E531E6C0111
:107D80007D01B7FF0CC082E090E0A82AB92AF094E8
:107D9000E094D094C094C11CD11CE11CF11CEFEB09
:107DA000FFEFAE22BF2221C020E430E0A22AB32A96
:107DB00038E73A8B80E1898BA2FE08C0F20180810E
:107DC0009181A281B38124E030E007C0F20180817B
:107DD0009181AA27BB2722E030E0420E531E6C019E
:107DE0007D018FEC9FEFA822B92287017601FE0169
:107DF0003196F88BEF87F9896F2E772488249924A0
:107E0000C801B701A40193010E941E416A3024F009
:107E10002A89620F615201C0605DEF85F889619324
:107E2000F88BEF87C801B701A40193010E941E419E
:107E300079018A01211531054105510509F7CC2445
:107E4000DD247601CE010196CF84C81AC501827364
:107E50009070892B19F0FE85F150FE87A6FE09C0AF
:107E60002989203111F482E001C081E03E85381B70
:107E70003E8728E0822E912C8A209B20A3FE18C0EA
:107E80008D85282F332727FD30958C2D9927821734
:107E900093073CF0E7EFFFEFAE22BF22882499243E
:107EA00007C0FD85FC19FD872E852F1B2E8703C07B
:107EB0003E853C193E87C50180789170892B69F415
:107EC0008E8506C0B10180E290E00E949340812F30
:107ED000182F11501816B4F31E87A1FE04C0B1016B
:107EE0008DE290E00BC0A4FE04C0B1018BE290E0F3
:107EF00005C0A5FE05C0B10180E290E00E9493405C
:107F0000A6FE10C0B10180E390E00E9493408989F1
:107F1000803141F4B101EA898E2F992787FD909530
:107F20000E949340B0FE0DC08E8506C0B10180E373
:107F300090E00E949340812F182F11501816B4F32F
:107F40001E87892869F02D8506C0B10180E390E085
:107F50000E949340212F122F11501216B4F31D8747
:107F600090E8692E712C6A207B20A7FC0DC08E85BD
:107F700006C0B10180E290E00E949340812F182F4B
:107F800011501816B4F31E87FA89F33641F4B10183
:107F90008C2D992787FD90950E94934045C02A8992
:107FA0002337B1F446015601198909C0F5018191C1
:107FB0005F01B101992787FD90950E949340115070
:107FC000A8F76401F989CF0ED11C2FEF298B2CC0A3
:107FD0003A89333519F00F8518891FC0460186018B
:107FE000B98808C0F8018491B10199270E94934093
:107FF0000F5F1F4FBA94FFEFBF16A1F764012989E5
:10800000C20ED11CF98B10C0F80182918F01B10111
:10801000992787FD90950E949340CE0101960817FD
:10802000190791F7188B0F876728B1F08E8506C066
:10803000B10180E290E00E949340812F182F1150EF
:108040001816B4F31E8708C0B101FA898F2F99273B
:1080500087FD90950E949340AA24BB2413C02A89CF
:10806000253241F43AE0398B1E861D8681E0A82E28
:10807000B12C08C0B101EA898E2F992787FD909510
:108080000E9493402B893C892F5F3F4F3C8B2B8B69
:10809000F101838183FF04C0EB89FC89F49103C063
:1080A000EB89FC89F081FA8B2A89222309F081CDA2
:1080B000F1018681978164960FB6F894DEBF0FBEFA
:1080C000CDBFDF91CF911F910F91FF90EF90DF9087
:1080D000CF90BF90AF909F908F907F906F905F9068
:1080E0004F903F902F900895FC0105900020E9F7F4
:1080F000809590958E0F9F1F0895FC01059061500B
:1081000070400110D8F7809590958E0F9F1F0895AD
:10811000FC016150704001900110D8F78095909556
:108120008E0F9F1F08950F931F93CF93DF938C01A2
:10813000EB018B81992781FF1BC082FF0DC02E812F
:108140003F818C819D812817390764F4E881F9818A
:108150000193F983E88306C0E885F985802F0995A6
:10816000892B31F48E819F8101969F838E8302C07B
:108170000FEF1FEFC801DF91CF911F910F9108956D
:1081800097FB092E07260AD077FD04D00CD006D025
:1081900000201AF4709561957F4F0895F6F7909539
:1081A00081959F4F0895AA1BBB1B51E107C0AA1FD1
:1081B000BB1FA617B70710F0A61BB70B881F991F88
:1081C0005A95A9F780959095BC01CD0108952F92FD
:1081D0003F924F925F926F927F928F929F92AF9257
:1081E000BF92CF92DF92EF92FF920F931F93CF93A4
:1081F000DF93CDB7DEB7CA1BDB0B0FB6F894DEBF3B
:108200000FBECDBF09942A88398848885F846E8460
:108210007D848C849B84AA84B984C884DF80EE80AA
:10822000FD800C811B81AA81B981CE0FD11D0FB6B3
:10823000F894DEBF0FBECDBFED010895A1E21A2E66
:10824000AA1BBB1BFD010DC0AA1FBB1FEE1FFF1FFA
:10825000A217B307E407F50720F0A21BB30BE40B4A
:10826000F50B661F771F881F991F1A9469F7609591
:108270007095809590959B01AC01BD01CF0108954B
:1082800054617267657420416371756973697469BB
:108290006F6E0000004C50493D20005250493D2077
:1082A000004C49523D20005249523D20004C534F52
:1082B0003D200052534F3D20004D6F74696F6E009A
:1082C00044657465637465642121212100546172E1
:1082D00067657420416371756972656400506F77DA
:1082E0006572696E672043616E6E6F6E2E2E2E0072
:1082F0004F424C49544552415445440046616C73C9
:108300006520416C61726D005374616E64696E67C3
:1083100020446F776E002564004F6F707321212118
:108320002121004F626C6974657261746F7200493B
:108330006E697469616C697A696E67212121003107
:1083400030205365636F6E64732E2E2E002039200B
:108350005365636F6E64732E2E2E00203820536594
:10836000636F6E64732E2E2E002037205365636F6B
:108370006E64732E2E2E002036205365636F6E645C
:10838000732E2E2E002035205365636F6E64732E7E
:108390002E2E0054657374696E67204C617365728C
:1083A000002034205365636F6E64732E2E2E0020E0
:1083B00033205365636F6E64732E2E2E002032209F
:1083C0005365636F6E64732E2E2E0020312053652B
:1083D000636F6E64732E2E2E00596F752042657484
:1083E0007465720052756E21212121000000000089
:0483F0000000000089
:00000001FF
